:046F24000100014225
:10698F00AF50055074D02FF582E4341DF583E5998F
:10699F00F022D3E5309400E52F94002290000FE011
:0369AF006403225C
:030003000256940E
:0B569400C0E0C083C082C0D075D00809
:10569F00852E82852D83E493FF201304C4540FFFBE
:1056AF00430FF08F80C284D28500C2870000D2875B
:1056BF00007580FF7580FEC284C28500C28700001E
:1056CF00D287007580FF30130CC213052EE52E70A4
:0956DF0006052D8002D213D2A8A9
:0956E800D0D0D082D083D0E03292
:03000B0002197661
:10197600C0E0C0F0C083C082C0D075D008758CD8D6
:10198600758A92D28C1242211262A6E531D3940056
:1019960040171531E53164056009E531640F6003D0
:1019A600021B88126BD4021B88753114E54ED39442
:1019B600004002154EE54FD394004002154FE53A1C
:1019C600D394004002153AE54BD394004002154BE0
:1019D600154CE54C123B441B7A001B4F011B27029A
:1019E6001AFF031A7C041A63051A4A061A31071AE3
:1019F600180819FF0900001B85D3E52C9400E52B78
:101A060094005003021B88E52C152C704D152B02F3
:101A16001B88D3E5379400E53694005003021B88F3
:101A2600E537153770021536021B88D3E548940052
:101A3600E54794005003021B88E5481548700215D7
:101A460047021B88D3E54A9400E5499400500302F7
:101A56001B88E54A154A70021549021B88D3E52AF8
:101A66009400E52994005003021B88E52A152A7084
:101A7600021529021B887885E6FF7003021B88EF92
:101A8600B40105900524801BEFB402101269A14031
:101A96002FE53015307002152F021B88EFB4030CAA
:101AA600900526E0F52FA3E0F5308028EFB4041268
:101AB6001269A1400BE53015307002152F021B8804
:101AC6008012EF64057003021B88EFB4060C752FB5
:101AD60002753058788506021B88EF64076003029A
:101AE6001B881269A1400BE53015307002152F02D4
:101AF6001B8878857600021B88D3E5399400E53883
:101B060094004008E539153970021538D3E53C9440
:101B160000E53B9400406BE53C153C7002153B80AC
:101B260061D3E5579400E55694004008E5571557EC
:101B360070021556D3E5559400E55494004043E5EC
:101B4600551555700215548039D3E5359400E534A2
:101B560094004008E535153570021534301423D34A
:101B6600E5339400E53294004018E53315337012DE
:101B76001532800EE551D39400400415518000754E
:0D1B86004C0AD0D0D082D083D0F0D0E03215
:03001300023EEFBB
:0D3EEF00C0E0C0F0C083C082C0D075D0100C
:103EFC00E545C394504003023FB0202303023FB07A
:103F0C00300C03023FB0E5A0540FF5587D077F013C
:103F1C00124ED65067202264E545700DE558B40C5E
:103F2C0008201005D210023FB020034A201047127F
:103F3C003FBB50047F0180027F0F126EB490000FC4
:103F4C00E0FF64016012EFB40302800C90000FE0FC
:103F5C00B40209123FBB50047F80801290000FE026
:103F6C00B4020E7D037F07124ED640057FA01200CF
:103F7C0016754202D20390053CE0F53A90002BE016
:103F8C00B5580D7D087F05124ED65004D2258014ED
:103F9C00053EE53EAE3D7002053D14F5828E83E58F
:043FAC0058F005457F
:103FB000D0D0D082D083D0F0D0E0327D037F071202
:033FC0004ED622B8
:030023000263B5C0
:1063B500C0E0C083C082C0D075D018309819C2988B
:1063C500E599B40A0812698F755000800AE550C333
:1063D5009490500312698F309902C299D0D0D0821F
:0563E500D083D0E0327E
:03003B0002492156
:0D492100C0E0C0F0C083C082C0D075D018C7
:10492E00C2CEE546C39410507C302479200C76AF6D
:10493E00A07804EF08800123D8FDF55953590F7D57
:10494E00077F02124ED65035202232E546700CE516
:10495E0059B40C07201204D212804A2004192012D6
:10496E001690000FE0B4020F7F0A126EB47F801211
:10497E000016754202D20490053CE0F53A90002BE9
:10498E00E0B5590D7D087F05124ED65004D2278012
:10499E00140540E540AE3F7002053F14F5828E834C
:0549AE00E559F005468B
:0B49B300D0D0D082D083D0F0D0E03212
:104B8000E4F55AF55B755C1E755DFF855B82855AA1
:104B900083E0F55E635EFFE55EF0E0655E60031254
:104BA0006F28635EFF855B82855A83E55EF0E06572
:104BB0005E6003126F28055BE55B7002055AE55DD8
:104BC000155D7002155CD3E55D9400E55C940050C2
:104BD000BA75985A758921758845758DE7758780EE
:104BE000758CD8758AEF75C90275C808753D1E7534
:104BF0003E60753F1E7540B075B701D2A9D2E8D2AC
:0F4C0000AA75C64C75EEFF75FEFFD2AF1266B3F4
:014C0F002282
:026F280080FEE9
:10696C00202E0F90053AE0F54EE54ED394004012E0
:10697C0080F7302E0D90053AE0F54FE54FD394009B
:03698C0050F9229D
:1069240030300AD214900024E04420800DC2147F39
:1069340008126EE8900024E054DFF0FD7F247E000E
:0469440012637F2239
:10300A008F70E57064017029202F047F018056209B
:10301A002F03023105123116400302310512311E07
:10302A00500C1231063014030231050230FB023013
:10303A00BBE57064027020202F047F028027202FB6
:10304A000302310512312640030231051269AB70C1
:10305A00030231050230D5E57064036003023105CD
:10306A00202F057F03026EE8302F24123116501FDD
:10307A00123126501A1269AB601512311E500B7F9D
:10308A000A12312E2014740230FB7F0302310230FF
:10309A002F2312313C501E7D017F02124ED640155D
:1030AA007D017F07124ED6500812310620144C803B
:1030BA00407F018043302F1712313C40127D017F3F
:1030CA0002124ED650091269AB60047F0280293081
:1030DA002F297D017F01124ED650201269AB701B39
:1030EA007D017F07124ED6500D7F0912312E201412
:1030FA000AD2300269247F01126EFB227F09126E06
:10310A00FB900536E0F532A3E0F533227D017F011D
:10311A00124ED6227D017F07124ED6227D017F02F2
:10312A00124ED622126EFB900536E0F532A3E0F578
:0A313A0033227D017F01124ED622E0
:104C1000C2957FFF126EE8124B807F071262DD5053
:104C20000512003E8003126063D28C7F081262DDA1
:104C300050051242E180FEC22A1268459000D1E080
:104C4000FF7C117D00125BDE125D5190000FE0B41D
:104C50000105122834801090000FE0FF6402600408
:104C6000EFB40303123271123D2E301D11E5427074
:104C70000DE52754A060077FA0126EB4C21D7D070A
:104C80007F05124ED64002C200E552C3940A50BBC3
:104C90003014B8E533453270B2C23012692480ABAB
:104A5700EF253EFFEE353DCF2401FDE43FFC22AFBD
:104A67005A7E00EF2403FDEE33FC22E53E255AF57E
:104A770082E4353DF58322E540255AF582E4353F4A
:104A8700F58322E56F256DF582E4356EF583E0FF4A
:104A9700E56F256DF582E4356EF58322E55A24022C
:104AA700FFE433FE22E56C2401FFE433FEC3E56D2A
:104AB7009FEE6480F874809822EF2540FFEE353F23
:104AC70022C2017FF47E01126C2AE56C25E0F56CA9
:104AD700756D0122E55C2EF582E4355BF583E0FD1B
:084AE70022753D1E753E6022A0
:106C2A00EF1FAA0670011ED39400EA9400400BE4F9
:0A6C3A00FDEDC394C850E90D80F78A
:016C4400222D
:10516D008F5BE55BB401197D017F06124ED6500CA5
:10517D009000B1E0FF7C0D7D00125BDE788506228C
:10518D00E55BB402131251DF50439000B2E0FF7C97
:10519D000D7D20125BDE8035E55BB404161251DF08
:1051AD00500C9000B4E0FF7C0D7D60125BDE7885C5
:1051BD00760622E55BB403197D027F06124ED650AA
:1051CD000C9000B3E0FF7C0D7D40125BDE788576A0
:0A51DD0001227D027F06124ED62249
:104ED600BF0107900020E0FE8048BF020790002136
:104EE600E0FE803EBF0307900022E0FE8034BF0450
:104EF60007900023E0FE802ABF0507900024E0FE0D
:104F06008020BF0607900025E0FE8016BF070790A9
:104F16000026E0FE800CBF0807900027E0FE800216
:104F2600E4FEBD0103EE1322BD0204EEA2E122BDA2
:104F36000304EEA2E222BD0404EEA2E322BD0504B0
:104F4600EEA2E422BD0604EEA2E522BD0704EEA20F
:074F5600E622BD0802EE3364
:014F5D002231
:101D9400124AE8900100E0F55A124A72E0123B44FC
:101DA4001DC3011DF8021E2D031E62041E97051E8D
:101DB400CC061F01071F31081F5D0900001F871291
:101DC4004A72A3E0B40A15E55A124AA5E545B507D7
:101DD4000BE4B506077D017F01021F45124A66E543
:101DE400456D7001EC6003021F87124A57C2287FB9
:101DF40001021F5A124A72A3E0B40A15E55A124AA4
:101E0400A5E545B5070BE4B506077D017F02021F72
:101E140045124A66E5456D7001EC6003021F8712A6
:101E24004A57C2287F02021F5A124A72A3E0B40A18
:101E340015E55A124AA5E545B5070BE4B506077D35
:101E4400017F03021F45124A66E5456D7001EC608F
:101E540003021F87124A57C2287F03021F5A124ADD
:101E640072A3E0B40A15E55A124AA5E545B5070B75
:101E7400E4B506077D017F04021F45124A66E54565
:101E84006D7001EC6003021F87124A57C2287F0459
:101E9400021F5A124A72A3E0B40A15E55A124AA55F
:101EA400E545B5070BE4B506077D017F05021F452F
:101EB400124A66E5456D7001EC6003021F87124A01
:101EC40057C2287F05021F5A124A72A3E0B40A15AA
:101ED400E55A124AA5E545B5070BE4B506077D01A9
:101EE4007F06021F45124A66E5456D7001EC6003EA
:101EF400021F87124A57C2287F06021F5A124A72CB
:101F0400A3E0B40A14E55A124AA5E545B5070AE464
:101F1400B506067D017F078028124A66E5456D7087
:101F240001EC705F124A57C2287F078029124A7257
:101F3400A3E0B40A0F124A72A3A3E070077D017FE5
:101F440008024E4B124A66E5456D7001EC7034127E
:101F54004A57C2287F0802100F124A72A3A3E070E6
:101F640022124A72A3E024F96008147016E4FF02F6
:101F74005EED7FF47E01126C2A7D5E7F021266891B
:031F84001242E125
:011F87002237
:101B9300753F1E7540B0900108E0F55A124A7EE089
:101BA300123B441BC5011BFD021C35031C6D041CA9
:101BB300A5051CDD061D15071D48081D7D09000030
:101BC3001D93124A7EA3E0B40A13124AA3E546B555
:101BD300070BE4B506077D017F01021D60AF5A12B2
:101BE3004A68E5466D7001EC6003021D93124AC01A
:101BF300124A5ED2287F01021D7A124A7EA3E0B404
:101C03000A13124AA3E546B5070BE4B506077D019F
:101C13007F02021D60AF5A124A68E5466D7001ECFF
:101C23006003021D93124AC0124A5ED2287F020249
:101C33001D7A124A7EA3E0B40A13124AA3E546B5FD
:101C4300070BE4B506077D017F03021D60AF5A123F
:101C53004A68E5466D7001EC6003021D93124AC0A9
:101C6300124A5ED2287F03021D7A124A7EA3E0B491
:101C73000A13124AA3E546B5070BE4B506077D012F
:101C83007F04021D60AF5A124A68E5466D7001EC8D
:101C93006003021D93124AC0124A5ED2287F0402D7
:101CA3001D7A124A7EA3E0B40A13124AA3E546B58D
:101CB300070BE4B506077D017F05021D60AF5A12CD
:101CC3004A68E5466D7001EC6003021D93124AC039
:101CD300124A5ED2287F05021D7A124A7EA3E0B41F
:101CE3000A13124AA3E546B5070BE4B506077D01BF
:101CF3007F06021D60AF5A124A68E5466D7001EC1B
:101D03006003021D93124AC0124A5ED2287F060264
:101D13001D7A124A7EA3E0B40A12124AA3E546B51D
:101D2300070AE4B506067D017F078031AF5A124AE0
:101D330068E5466D7001EC7057124AC0124A5ED2D4
:101D4300287F078032124A7EA3E0B40A13124AA303
:101D5300E546B5070BE4B506077D017F08024E4B48
:101D6300AF5A124A68E5466D7001EC7023124AC0FF
:101D7300124A5ED2287F0802100F124A7EA3A3E004
:101D8300700E124A7EA3E024F870057F01125EED07
:011D9300222D
:0447D4008C5B8D5C11
:1047D800055CE55C7002055B14F5828C83E0F9707A
:1047E8000302487BEF7005124AE88009BF0106758D
:1047F8003F1E7540B0302846EF7007E965456002F6
:10480800C322BF0107E965466002C322E4FEEEC386
:10481800995029EF700F124ADBE53E2E124A76E0D6
:104828006D6002C322EF6401700F124ADBE5402E6F
:10483800124A82E06D6002C3220E80D2D322202861
:1048480033E4FEEEC3995029EF700F124ADBE53EC0
:104858002E124A76E06D6016C322EF6401700F12C3
:104868004ADBE5402E124A82E06D6002C3220E80C8
:04487800D2D322C3B2
:01487C002219
:06100F008F5BAB05AA0493
:101015007D027F07124ED65011E55BB4050C8B821D
:101025008A83E06405700302127C7D017F07124EFE
:10103500D65011E55BB4050C8B828A83E06406709B
:101045000302127CC229EB24FFF582EA34FFF58303
:10105500E0F55D8B828A83E0FFF55EA3E0F9F55F3D
:10106500EF123B44108501108C02109303109A0473
:1010750010A10510A80610AF0710B608000010BB98
:10108500755C01D229802F755C02D2298028755C98
:1010950004D2298021755C08D229801A755C10D28A
:1010A500298013755C20D229800C755C40D229807B
:1010B50005755C80D229E924FE700302117D24F8B0
:1010C500605C2409600302118FE55BB401059000A3
:1010D500208045E55BB40205900021803BE55BB4CB
:1010E50003059000228031E55BB404059000238060
:1010F50027E55BB40505900024801DE55BB4060576
:101105009000258013E55BB407059000268009E56E
:101115005B64087077900027E0455CF0806EE55BC6
:10112500B401059000208045E55BB40205900021DF
:10113500803BE55BB403059000228031E55BB40498
:10114500059000238027E55BB40505900024801DEC
:10115500E55BB406059000258013E55BB4070590B3
:1011650000268009E55B64087022900027E0FFE512
:101175005CF4FEEF5EF08014E55BB4050D8B828AAE
:1011850083E0FFD22E122995C229C2292029030204
:10119500127CE55BB40109900020E0FD7F208060B2
:1011A500E55BB40209900021E0FD7F218052E55BFB
:1011B500B40309900022E0FD7F228044E55BB4047E
:1011C50009900023E0FD7F238036E55BB405099097
:1011D5000024E0FD7F248028E55BB4060990002506
:1011E500E0FD7F25801AE55BB40709900026E0FD48
:1011F5007F26800CE55BB4080C900027E0FD7F2777
:101205007E0012637F126D3DD2AF2028047F0180DE
:10121500027F02126EFBA228922E12696CAD5DE46C
:10122500FF126689AD5EE4FF126689E55FB40104CD
:101235007D388007E55FB40A077D367F061266892B
:10124500E55BB405031264E37D077F05124ED650B6
:101255000A200007C22F7F0312300A7D017F011289
:101265004ED64005C22F12300A7D017F02124ED69E
:071275004005C22F12300AF0
:01127C00224F
:024E4B008F5B7B
:104E4D00ED24FF922E12696CE55B123B444E760108
:104E5D004E7B024E80034E85044E8A054E8F064EC4
:104E6D0094074E990800004E9F90002080219000DD
:104E7D0021801C9000228017900023801290002426
:104E8D00800D90002580089000268003900027E07B
:104E9D00F55CE55C6024755E01E4F55DE55C30E094
:104EAD0007AD5EE4FF126689E55CC313F55C055E34
:104EBD00055DE55DC3940840E3227D187F0212660F
:084ECD00897D537F0212668902
:014ED50022BA
:1062DD00C2AFD284C285BF070BC28600E580A2E2A1
:1062ED0092298019BF080BC28600E580A2E392298E
:1062FD00800BBF0508C28600E580139229D286D295
:05630D0085D2AFA229BA
:016312002268
:1045C700C228D22CE4FF1259BD7D2E7F03126689C3
:1045D7007D607F021266897F03126EE83023FD201B
:1045E70023FDE5456407703B7E017F50124AE88F43
:1045F700828E837407F07D01E53E2D124A76E582AF
:1046070024FFF582E58334FFF583E0F9EF2DF5828A
:10461700E43EF583E9F00DBD08DED2287F647E0015
:10462700126C2A7F081262DD5043302895D22CE4A1
:10463700FF1259BD7D607F021266897D327F0612A7
:1046470066897D1E7F05126689C22CE4FF1259BD5B
:104657007C017D507B087F507E011255097F08122F
:1046670062DD50097F327E00126C2A80F07F647E03
:0446770000126C2A97
:01467B00221C
:0254A0008F5A21
:1054A200900138E0F55BE55A7020E55B124AA5E50C
:1054B200456F7001EE704F7460255BF582E4341E17
:1054C200AF82F55D8F5E7F408024E55A64017036BD
:1054D200E55B124AA5E5466F7001EE702974B025AE
:1054E2005BF582E4341EAF82F55D8F5E7F101200A1
:1054F20016855E82855D83E0FFA3E0FD126DA18FBC
:065502005CE4FD124F5EA7
:015508002280
:024F5E008D6B59
:104F600075F020EF900280123B38AF8285836E8F00
:104F70006FE0F56CD394004060E56C9410505AE5F6
:104F80006B7014124ACA124AAC504E124A8A124F1F
:104F9000DF056D056D80EFE56B64017019124AC87D
:104FA000124AAC5034124A8A124FDF302302802951
:104FB000056D056D80EAE56B6402701D124AC8122A
:104FC0004AAC5015124A8AA3E0FD12651330230340
:0E4FD000024D2F056D056D80E67F50126EB408
:084FDE0022A3E0FD126513227D
:100A5400855C82855B83A3A3E0FF855C82855B83E1
:100A6400A3222430F58274003EF583EDF0AF62EFEB
:100A74003395E0FEE55F2FF582E55E3EF583A3A3A3
:100A8400E0FF126D7CAD07AF63EF3395E0FEEF221C
:100A9400A3A3E0FFE55C2404F582E4355BF583E081
:100AA40022E55F2405F582E4355EF583E022E55F07
:100AB4002405F582E4355EF583E0FFE55F2406F561
:100AC40082E4355EF583E0222431F58274003EF53C
:100AD40083EDF0AF62EF3395E0FEE55F2FF582E53D
:100AE4005E3EF583222455F582E4340AF583EFF063
:100AF400E56275F007A422E562FD3395E0FCE55F4D
:100B04002DF582E55E3CF583E0FFE55F2DF582E59A
:100B14005E3CF583228E69F56AAF68EF3395E0FE9B
:100B2400E5662FF582E5653EF58322ECFF3395E01B
:100B3400FEEF25E0FFEE33FE75F020ED123B38E5C5
:100B4400822FF582E5833EF58322A3A3A3E0FF8DE4
:100B5400828C83E5822404F582E43583F58322E5DF
:100B6400662405F582E43565F583E022E55E75F0DB
:100B740007A42454F582E4340AF58322E55E75F073
:100B840007A42451F582E4340AF5832224E0F58293
:100B9400740A3EF583E5822DF582E5833CF58322D4
:100BA400E55E75F007A42453F582E4340AF5832244
:100BB400E55F2405F582E4355EF583E0FFE55F2417
:100BC40006F582E4355EF583E022E55E75F007A460
:100BD4002452F582E4340AF58322749F2562F58257
:100BE400E43400F58322746F2562F582E43400F561
:100BF40083222450F582E4340AF58322E560240537
:100C0400F582E4355FF58322D3EF6480948022ABD0
:100C140007AA068B828A83A3A3A3E0FFEB2404F52F
:100C240082E43AF583E0FD228F828E83A3A3A3E0BE
:100C340022855F82855E83A3A322AB5DAD5AAF5C40
:100C4400AE5B2233CE33CE92E022A2E0CE13CE139B
:100C54002275F00AA42DFDE5F03CFCE56622E56072
:100C64002405F582E4355FF583E022E56275F0083A
:100C740090015822E55E75F007A42455F582E4340A
:100C84000AF583E022AB5AAD5DAF5CAE5B22EF7C2C
:100C9400002563FDEC35628D82F58322A3A3E0FF7A
:100CA400AD5A22E5662DF582E5653CF583A3A322C2
:100CB400540FF5657808AF03AE02EF08220564E52A
:100CC40064AE632225E0FFEE33FE75F020E5642276
:100CD40075F020123B38E0FEA3E0FF22E0FAA3E027
:100CE400FB780CFFAE020822E0FCA3E0FD7804FFD1
:100CF400AE040822E5632561F582E43562F58322BA
:100D0400E5662DF582E5653CF58322E5662FF582DF
:100D1400E5653EF583222480F58274023EAF82228B
:100D24002560F560E4355FF55F22856082855F8329
:0B0D3400228F828E83A3A3E0640A22BA
:02055B008F5AB5
:10055D00C229E4F542D222D22C1259BD7D4B7F0225
:10056D001266897D02E4FF1266897D32E4FF126610
:10057D00897D607F021266897D027F07124ED650FB
:10058D00057F04126EE8900528E0F536A3E0F537F7
:10059D007F03126EE8E55A7006A22392288009E5C2
:1005AD005AB40104A2249228E53745367005D229A4
:1005BD00020A223028DFE55A7006A223922880090C
:1005CD00E55AB40104A22492282028EAE55A700BBA
:1005DD00755B1E755C6085455D800EE55AB401093D
:1005ED00755B1E755CB085465DE55DD3940050036B
:1005FD00020A1C855C82855B83E0640B6003020A42
:10060D0017A3E0FFB40A0AE55DB40205D229020A78
:10061D001CEF6401701E120A5EA3E0640A7015E5FA
:10062D005D6405700F120A5E120A94120A4D1231A2
:10063D0044020A1C120A5EE0B40111120A5EA3E024
:10064D00B40109120C3E121732020A1C120A5EE0A6
:10065D006401701E120A5EA3E064027015E55D640C
:10066D0005700F120A5E120A94120A4D12618C0265
:10067D000A1C120A5EE06401701D120A5EA3E0649A
:10068D00037014E55DB4050F120A5E120A94FDABFA
:10069D005A1237B0020A1C120A5EE0B4011D120A8A
:1006AD005EA3E0B40415E55DD39405400EAB5AADE1
:1006BD005CAC5BAF5D122D91020A1C120A5EE06408
:1006CD0001701D120A5EA3E064057014E55DB405AA
:1006DD000F120A5E120A94FDAB5A125AAF020A1C8F
:1006ED00120A5EE06401701D120A5EA3E0640670DA
:1006FD0014E55DB4050F120A5E120A94FDAB5A1291
:10070D004DBE020A1C120A5EE0B4011D120A5EA360
:10071D00E0B40715E55DD39405400EAB5AAD5CAC66
:10072D005BAF5D124511020A1C120A5EE064017096
:10073D001D120A5EA3E064087014E55DB4050F1286
:10074D000A5E120A94FDAB5A126349020A1C120A80
:10075D005EE0B40215120A5EA3E0B40A0DE55DB4C5
:10076D000308AF5A126313020A1C120A5EE0B402A8
:10077D0016120A5EA3E0B4010EE55DB40E09120C6B
:10078D0040122ECE020A1C120A5EE0B40216120AA4
:10079D005EA3E0B4020EE55DB40709120C401252DF
:1007AD00DA020A1C120A5EE0B40215120A5EA3E018
:1007BD00B4090DE55DB40308AF5A125434020A1C96
:1007CD00120A5EE064027019120A5EA3E0B4091108
:1007DD00E55DB4040C120A5E120CA0126758020AF1
:1007ED001C120A5EE064037021120A5EA3E0640A23
:1007FD007018E55D64057012120A5E120A94FD12FE
:10080D006DA1AD5A124729020A1C120A5EE064035B
:10081D007029120A5EA3E064017020E55DD3940592
:10082D004019120A5E120A94FD126DA1855A62AB2F
:10083D005DAD5CAC5B123E0F020A1C120A5EE064F9
:10084D00037021120A5EA3E064027018E55D640571
:10085D007012120A5E120A94FD126DA1AD5A125F4A
:10086D006D020A1C120A5EE0B40315120A5EA3E0C3
:10087D00B4030DE55DB40308AF5A125FE9020A1C1B
:10088D00120A5EE0B40318120A5EA3E0B40410E588
:10089D005DD394034009120C891249BE020A1C1241
:1008AD000A5EE0B40315120A5EA3E0B4050DE55D22
:1008BD00B40308AF5A126D8F020A1C120A5EE0B41F
:1008CD000316120A5EA3E0B4060EE55DB405091227
:1008DD000C4012686B020A1C120A5EE06403701968
:1008ED00120A5EA3E0B40711E55DB4040C120A5EB2
:1008FD00120CA0126B9A020A1C120A5EE0B40316C7
:10090D00120A5EA3E0B4080EE55DB40409120C40B2
:10091D00126890020A1C120A5EE064057014E55D0F
:10092D00B4040F120A54A3A3E0FDAB5A121F8802A0
:10093D000A1C120A5EE0B40516120A98B40B10E5F3
:10094D005DD394054009120C8912339D020A1C12C5
:10095D000A5EE064067014E55DB4040F120A54A338
:10096D00A3E0FDAB5A12217A020A1C120A5EE0B412
:10097D000616120A98B40B10E55DD39405400912C2
:10098D000C891226AB020A1C120A5EE06409701A69
:10099D00120A5EA3E0B40A12E55DB4040D120A5EFC
:1009AD00A3A3E0FF125D9A020A1C120A5EE064091D
:1009BD007018120A5EA3E0B40110E55DB4040B12C9
:1009CD000A5E120CA012626F8045120A5EE0B40935
:1009DD0017120A5EA3E0B4020FE55DD3940440083C
:1009ED00120C3E1214EB8027120A5EE06409701A95
:1009FD00120A5EA3E0B40310E55DB4040B120A5EA7
:100A0D00120CA0125D0880078000AF5A126BB72040
:100A1D0029030205A2C21DD22CAF5A1259BD7D6009
:100A2D007F021266897D327F031266897F03126E03
:0F0A3D00E8125DE27FFF126EB4E47885F6C22204
:080A4C0022FD126DA1AD5A223A
:081732008E5E8F5F8D608B61FC
:10173A00120C2CFFE55F2404120AA9FD12641E8F05
:10174A006274E22562F562C394005003021933E51C
:10175A006294144003021933E5616406701D120A8B
:10176A00A5B4010C120AF4120BF67401F002192F37
:10177A00120AF4120BF6E4F002192FE561640E6006
:10178A0003021851E55F240C120AA9FFB40A14E5F2
:10179A005F240D120AA9B40A0A120AF4120B86E48B
:1017AA00F08013E55F240D120AA9FD126C0E120ACD
:1017BA00F4120B86EFF0E55F240A120AA9FFB40AB5
:1017CA0014E55F240B120AA9B40A0A120AF4120BCE
:1017DA00D4E4F08013E55F240B120AA9FD126C0E03
:1017EA00120AF4120BD4EFF0E55F2409120AA9FFDA
:1017FA00640A6006EFD39409400A120AF4120BAA8B
:10180A00E4F08010E55F2409120AA9FF120AF41213
:10181A000BAAEFF0120AA5FFB40B15E55F24061216
:10182A000AA9B40B0B120AF4120B7674FFF08008A3
:10183A0012195F120B76EFF012193B120AE9120B1A
:10184A00F67401F002192FE561640A706E120AF447
:10185A00120B86E4120AF3120BD4E4F0E55F2409B2
:10186A00120AA9FF640A6006EFD39409400A120A11
:10187A00F4120BAAE4F08010E55F2409120AA9FF0A
:10188A00120AF4120BAAEFF0120AA5FFB40B15E51F
:10189A005F2406120AA9B40B0B120AF4120B76740F
:1018AA00FFF0800812195F120B76EFF012193B1243
:1018BA000AE9120BF67401F002192FE56164097046
:1018CA0068120AF4120B86E4120AF3120BD4E41219
:1018DA000AF3120BAAE4F0120AA5FFB40B15E55F8E
:1018EA002406120AA9B40B0B120AF4120B7674FF1F
:1018FA00F08013E55F2406120AA9FD126C0E120A83
:10190A00F4120B76EFF0E55F2407120AA9FFE55FF0
:10191A002408120AA9FD126C0E120AF4120AE9121C
:10192A000BF67401F0D22B8002C22BAF60126E8AC2
:10193A0022E55F2407F582E4355EF583E0FFE55F83
:10194A002408F582E4355EF583E0FD126C0EE5624B
:10195A0075F007A422E55F2406F582E4355EF58377
:0C196A00E0FD126C0EE56275F007A4228F
:103144008F5E8D5FE55ED3941D5003023250E55EC1
:1031540094324003023250D22CAF5F1259BD7D46E7
:103164007F07126689AF5E1234C574E2255EF55E90
:10317400120B82E07021120BCEE0701B120BA4E044
:103184007015120B70E0700F120C78700A1232690D
:103194007D537F02023246123258E55E75F007A471
:1031A400120BF6E070047D3680027D387F061266CD
:1031B40089123258120B80E0FFD394014034EF940B
:1031C40013502F7D097F06126689120B801232601C
:1031D4007FF47E01126C2A7D0E7F031266897D3591
:1031E4007F061266897D097F06126689120BCE124C
:1031F40032607FF47E01126C2A120BA4E0FF60059A
:10320400125A60800A1232697D0F7F031266897D2B
:10321400277F02126689120B70E0FFF46008126CBB
:10322400AF1234C580077D187F021266897D377F0F
:1032340004126689120C78FF126CAF1234C57D0536
:103244007F06126689C22CAF5F0259BDC22BAF5FE5
:10325400126E8A227FF47E01126C2A22E0FF126C25
:0D326400AF1234C5227D187F021266892248
:02618C008D5E26
:10618E00EFD3941D402AEF9432502574E22FFFE492
:10619E00FEEEFD3395E0FCEF75F007A42450F5827A
:1061AE00E4340A120B97E4F00EBE07E5D22B800200
:0761BE00C22BAF5E126E8AD6
:0161C50022B7
:062ECE008E5E8F5F8D6037
:102ED400D22A120C2CFFE55F2404120AC3122FF528
:102EE400C39418501C855F82855E83A3A3A3E0FF6F
:102EF400E55F2404120AC3FD126D697883A6078076
:102F040006E47883F6C22A120AB2122FF5C3943C5F
:102F1400500D120AB2FD126D697884A6078006E48A
:102F24007884F6C22AE55F2407120AC3FF126E1CD6
:102F34008F61E561D394004017E56194085011E571
:102F44005F2407120AC3FF126E1C7880A60780064E
:102F540078807601C22AE55F2408120AC3FFE55F80
:102F64002409120AC3122FFE401FE5619420501950
:102F7400E55F2408120AC3FFE55F2409120AC3FDB2
:102F8400126D697888A607800678887601C22AE5DA
:102F94005F240A120AC3FFE55F240B120AC3122F2F
:102FA400FE401FE561940D5019E55F240A120AC31F
:102FB400FFE55F240B120AC3FD126D697881A60731
:102FC400800678817601C22AE55F240C120AC3FFC9
:102FD400E55F240D120AC3FD126D697882A60730DD
:102FE4002A071257A9D22B8002C22BAF60126E8A15
:102FF40022FD12641E8F61E56122FD12641E8F6141
:06300400E561D3940022F7
:0652DA008E5E8F5F8D6007
:1052E000D22A120C2CFFE55F2404120BC512534581
:1052F0009418501C855F82855E83A3A3A3E0FFE51D
:105300005F2404120BC5FD126D697883A607800621
:10531000E47883F6C22A120BB4125345943C500D24
:10532000120BB4FD126D697884A6078006E47884B8
:10533000F6C22A302A071257A9D22B8002C22BAFFD
:0453400060126E8AFF
:0B53440022FD12641E8F61E561C32290
:106E1C00120C0C4008EF6480948A5001227F0022EF
:106D6900AE05126E1CEFC454F0FDAF06126E1CEF97
:036D79004DFF22A9
:106313008F5ED22C1259BD7D1E7F081266897D26A1
:106323007F081266897D527F04126689C22A126829
:1063330045125C747880E6FF125A60125967C22CCA
:06634300AF5E1259BD22FD
:106758008D5EEFD3940A4006EFD3940F4003EF7099
:106768000E90002BEFF0D22BAF5E126E8AD322C2AE
:086778002BAF5E126E8AC322F2
:025434008F5E89
:10543600D22C1259BD7D207F051266897D2E7F03F1
:105446001266897D527F0412668990002BE0F55F13
:10545600E55FB40B067D5F7F078034E55FB40C061D
:105466007D5E7F068029E55FB40D067D0A7F02809A
:105476001EE55FB40E067D327F028013E55FB40F32
:10548600067D467F028008E55F70077D0A7F03126E
:095496006689C22CAF5E1259BDFB
:01549F0022EA
:106B9A008D5E120C0C400EEF6480948650071263CF
:0D6BAA00EAD22B8002C22BAF5E126E8A224F
:02686B008D5E40
:10686D00120C1312641E120C0C4010EF648094A1D4
:10687D005009900029EFF0D22B8002C22BAF5E128F
:02688D006E8A11
:01688F0022E6
:026890008D5E1B
:10689200120C1312641E120C0C4010EF648094A1AF
:1068A2005009900028EFF0D22B8002C22BAF5E126B
:0268B2006E8AEC
:0168B40022C1
:106D7C00D3EF648094814008EF64809489500122A1
:036D8C007F002263
:106E2C00120C0C4008EF648094A15001227F0022C8
:0814EB008E5E8F5F8D608B6146
:1014F300120C2C14F56374FC2561F5616403600F11
:10150300E56164076009E561640B60030216CDC3FE
:10151300E5636480948050030216CDE56364809490
:101523008840030216CDE4F562120A8B7803C333B5
:10153300CE33CED8F92430F58274003EF583AF6202
:10154300EF3395E0FE120B43E4F00562E562B40865
:10155300D8756204E56164037027120AFB12172829
:10156300120A897803C333CE33CED8F9120A6678C8
:1015730003C333CE33CED8F92431F5827400021677
:10158300C4E5616407705D120AFB121728120A8909
:101593007803C333CE33CED8F9120A667803C33344
:1015A300CE33CED8F9120ACCA3120A827803C333FE
:1015B300CE33CED8F91216D5C333CE33CED8F924D1
:1015C30033F5827400120AD2E5822406120B5B12F1
:1015D3000A847803C333CE33CED8F92434F5827426
:1015E300000216C4E561640B60030216CD120AFB08
:1015F300A3E0FD12641E126E2C120A897803C33312
:10160300CE33CED8F9120A667803C333CE33CED89D
:10161300F9120ACCA3120A827803C333CE33CED88D
:10162300F91216D5C333CE33CED8F92433F58274E9
:1016330000120AD2E5822406120B5B120A84780395
:10164300C333CE33CED8F92434F5827400120AD2D0
:10165300E5822407120B5B120A847803C333CE336B
:10166300CED8F92435F58274003EF583EDF0E562BA
:10167300FD3395E0FC120B0EE5822408F582E43578
:1016830083120B0AE5822409120B5BE0FD12641E30
:10169300126E2C120A897803C333CE33CED8F924C1
:1016A30036F5827400120AD2E582240A120B5B1209
:1016B3000A847803C333CE33CED8F92437F5827442
:1016C300003EF583EDF0D22B8002C22BAF60126E89
:0116D3008A8C
:1016D400222432F58274003EF583EDF0E562FD3399
:1016E40095E0FCE55F2DF582E55E3CF583E582241B
:1016F40004F582E43583F583E0FFE55F2DF582E5AB
:101704005E3CF583E5822405F582E43583F583E0C8
:10171400FD12641E126E2CAD07AF63EF3395E0FE2D
:0E172400EF780322A3E0FD12641E126E2C2249
:045D08008D5EAC07F9
:105D0C00D3EC648094804035EC64809489502EE40C
:105D1C00FDECFF3395E0FEEF7803C333CE33CED8E2
:105D2C00F92428F58274003EF583EDFF3395E0FEEF
:105D3C00120B43E4F00DBD08D8D22B8002C22BAF5E
:045D4C005E126E8AEB
:015D50002230
:10626F008D5E120C0C402FEF648094895028EF1430
:10627F00FFE55E24FF922A124FE6D22CAF5E125931
:10628F00BD7542017F327E00126C2AE54270FCC25E
:07629F002CAF5E1259BD2275
:084511008F5E8C5F8D608B61F1
:10451900856082855F83120B4EE0FD12641E8F62F7
:10452900E562D3940050030245BFE562943240032B
:104539000245BFE55E64067036D22CAF611259BDE3
:104549007D527F05126689AF621234C5120C62B4BE
:10455900010A120BDE7401F07D388007120BDEE4CC
:10456900F07D367F06126689C22CAF610259BDE51E
:10457900602406120C66640B703C120C62B40108CC
:10458900120BDE7401F08005120BDEE4F074F925DC
:104599005EF55E75F004123A7EAFF0EF7014E560D7
:1045A9002406FBE4355FFAAD62E4FF1236BBD22B79
:0D45B9008006C22B8002C22BAF61126E8AF9
:0145C60022D2
:082D91008F5E8C5F8D608B6189
:102D9900856082855F83120B4EE0FD12641E8F628F
:102DA900E562D394005003022EC6E56294284003DD
:102DB900022EC6E55E64067037D22CAF611259BD8A
:102DC9007D527F05126689AF621234C5120C00E08C
:102DD900B4010A120BEA7401F07D388007120BEA7C
:102DE900E4F07D367F06126689C22CAF610259BDB7
:102DF900E5602406120C04E0640B6003022EC6127F
:102E09000C00E0B40108120BEA7401F08005120B02
:102E1900EAE4F0E4FFFEE5602407120C04E5822EE3
:102E2900120B5BE0B40B04AF0680040EBE08E7EF9B
:102E39007003022EC6C394084003022EC6120C6FFB
:102E4900123B38EFF07E01EF2401FDE433FCEEC3C1
:102E59009DEC6480F87480985020E5602406120C7B
:102E690004E5822E120B5BE0FD120C6F123B38E574
:102E7900822E120B5BEDF00E80CDE5602408120C5A
:102E890004E5822F120B5BE0640B602DEF2408FE32
:102E9900C3E55E9EF55E75F004123A7EAEF0EE7003
:102EA9001CE5602407FDE4355FFC7E00ED2FFBEE99
:102EB9003CFAAD627F011236BBD22B8002C22BAF26
:042EC90061126E8A9A
:012ECD0022E2
:0836BB008F638D648A658B6644
:1036C300756801E4F567120B1DE0FF64097037129A
:1036D30037A18003120C47D8FB120B1912379378CA
:1036E30008EF088003120C47D8FB8E69F56AE5687A
:1036F300FD3395E0FC120CA7E0FF120CA7A3E0FD3D
:10370300126DA1023750120B1DE0FF1237A1800387
:10371300120C47D8FB120B191237937804EF088069
:1037230003120C47D8FB120B19A3A3E0FF126EDEA2
:10373300EF426AAE69AF6A7804EF088003120C4760
:10374300D8FB120B19A3A3A3E0FF126EDEEF426AAC
:10375300E563700DAF67120A8D120CC8900AC08022
:1037630010E563B40115AF67120A8D120CC89005FA
:1037730030120B40E569F0A3E56AF074042568F59F
:0F378300680567C3E5676480949050030236C9F8
:1037920022A3E0FF126EDEEF426AAE69AF6A221226
:0E37A2006EDE7569008F6AAE697804EF08224A
:0A6EDE00EFD3940940037F00222245
:0237B0008B5E2E
:1037B20012641E8F61E561D394005003023899E5CB
:1037C2006194334003023899D22CAF5E1259BD7D09
:1037D200527F05126689AF611234C5746F2561127A
:1037E2000BEEE060047D3880027D367F061266892A
:1037F2007F2C7E01126C2AE561120C71123B38E0BB
:10380200F55F70077D1B7F061266897D577F021266
:103812006689E55F603F756001AF5F120A8D240122
:10382200FFE43EFEAD60ED3395E0FCC3ED9FEE6438
:1038320080F8EC648098501DAF60EF3395E0FE7520
:10384200F008E561900158120B40E0FDE4FF1266BA
:1038520089056080C47F2C7E01126C2AE561900587
:1038620030120CD4900000EEF0A3EFF04E70077D02
:103872001B7F061266897D0C7F0312668990000009
:10388200E07002A3E06009E56114FD7F01122AF3F2
:0E389200C22CAF5E0259BDC22BAF5E126E8A11
:0138A0002205
:024DBE008B5E0A
:104DC00012641E8F5FE55FD394004077E55F9433F4
:104DD0005071D22CAF5E1259BD7D527F051266898B
:104DE000AF5F1234C5749F255F120BE2E060047D53
:104DF0003880027D367F061266897F2C7E01126C18
:104E00002A7F2C7E01126C2AE55F900AC0120CD416
:104E1000900000EEF0A3EFF04E70077D1B7F0612AE
:104E200066897D0C7F03126689900000E07002A302
:104E3000E06009E55F14FDE4FF122AF3C22CAF5EC7
:0A4E40000259BDC22BAF5E126E8A4C
:014E4A002245
:026349008B5E69
:10634B0012641EAD07EDD394004021ED9433501C25
:10635B00E4FC900AC0120B2FE4F0A3F00CBC10F27B
:10636B00749F2D120BE2E4F0D22B8002C22BAF5E96
:03637B00126E8A15
:01637E0022FC
:025AAF008B5E0C
:105AB10012641EAD07EDD394004038ED943350339A
:105AC100E4FC900530120B2FE4F0A3F00CBC10F2B3
:105AD100746F2D120BEEE4F0FCECFF3395E0FE75D4
:105AE100F008ED900158120B40E4F00CBC08EAD22A
:0A5AF1002B8002C22BAF5E126E8AFA
:015AFB002288
:042AF3008F628D63FE
:102AF700E4F564E5627052AF64120A8D25E0FDEEDD
:102B070033FCAF63120A8D7805C333CE33CED8F9C1
:102B1700120B90120CE08003120C4ED8FB120CB46F
:102B27008003120C4ED8FB540FF566AF63120A8D63
:102B37007805C333CE33CED8F9120B90120CEC8044
:102B470003120C4ED8FB022BB1E56264017064AF2F
:102B570064120A8D25E0FDEE33FCAF63120A8D780F
:102B670005C333CE33CED8F92450F5827405120B42
:102B770096120CE08003120C4ED8FB120CB48003A3
:102B8700120C4ED8FB540FF566AF63120A8D780509
:102B9700C333CE33CED8F92450F5827405120B9681
:102BA700120CEC8003120C4ED8FB540FF567ED5452
:102BB7000FF568E565700CE5667008E5677004E574
:102BC70068607CAD65E4FF126689AD66E4FF126656
:102BD70089E56564097045856769AF69FE7804EF23
:102BE700088003120C47D8FBF569E5684269E56977
:102BF700B4990B7D09E4FF1266897D098027E56991
:102C070075F00A84F56AFDE4FF126689E56A75F0D6
:102C17000AA4FFC3E5699FF56AFD8009AD67E4FF74
:102C2700126689AD68E4FF1266897FF47E01126C33
:0F2C37002A0564C3E564648094A05003022AFA5E
:012C4600226B
:10641E00EFD394004015EF940B5010EFC3940A5035
:10642E0008EF75F00AA4FE8002E4FEEDD39400405E
:10643E000EED940B5009EDC3940A5003ED2EFEAFF2
:01644E000647
:01644F00222A
:0649BE008E5E8F5F8B602E
:1049C400756105756240D3ED64809484407CED6428
:1049D4008094A55075ED24FDF563D39404406BE5F4
:1049E4006320E06613F5640562E562AE617002055A
:1049F4006114F5828E83E564F07403255FF55FE44A
:104A0400355EF55EE4F563E563C395645033855F15
:104A140082855E83E0FFA3E0FD126DA10562E5627D
:104A2400AC617002056114F5828C83EFF0055FE5DB
:104A34005F7002055E055FE55F7002055E056380D9
:104A4400C6D22BAF60126E8AD322C22BAF60126E15
:024A54008AC313
:014A5600223D
:043E0F008C5F8D60D7
:103E1300120C0C5003023EE7EF64809495400302BA
:103E23003EE7EB648094875003023EE7EB648094A3
:103E3300E44003023EE7120A8D7805C333CE33CE46
:103E4300D8F9120D1AF5638F64EB24FBF565D3944F
:103E5300025003023EE7E56575F00384E5F0600375
:103E6300023EE7E56575F00384F567C3941050746B
:103E7300120CC17002056314F5828E83E567F0743A
:103E830005120D24E4F565E565C395675052120DDF
:103E93002EE0F566B40A10120CC17002056314F526
:103EA300828E83E4F0800F120CC17002056314F557
:103EB300828E83E566F0120D2EA3E0FF120D2EA372
:103EC300A3E0FD126DA18F66120CC170020563148D
:103ED300F5828E83E566F07403120D24056580A7D1
:0B3EE300D22B8002C22BAF62126E8A4D
:013EEE0022B1
:0826AB008E5E8F5F8D608B6174
:1026B300C22A120D35600302274812282350030251
:1026C3002743E5649408E56394075074C3E56064A5
:1026D30080948A506B120C35A3E0F562B401069026
:1026E3000520022798E562B4020690052202279886
:1026F300E562B40306900524022798E562B4040654
:10270300900526022798E562B4050690052802275E
:1027130098E562B4060690052A022798E562B40795
:102723000690052C022798E562B4080590052E80D3
:1027330064E562B40905900530805AD22A02281450
:10274300D22A022814120C35E064017052AD60AF36
:102753005FAE5E1228235003022814E5649408E553
:102763006394074003022814C3E5606480948A409D
:1027730003022814120C35A3E0F562B40A05900590
:10278300328012E562B401059005348008E562B435
:102793000209900536E563F0A3806FD22A80721296
:1027A3000C35E06402706AAD60AF5FAE5E125B48E9
:1027B3007563008F64C3E5649463E56394005051CB
:1027C300C3E560648094885048120C35A3E0F56239
:1027D300B40107900538EFF08037E562B402059045
:1027E30005398026E562B4030590053A801CE5624D
:1027F300B4040590053B8012E562B4050590053CE1
:102803008008E562B4060890053DE564F08002D2D5
:0F2813002A302A04C22B8002D22BAF61126E8AA8
:102822002212487D8E638F64D3E564943BE5639402
:02283200002282
:06487D008E658F66A9059F
:104883007D057C00120D04E0C3940A4005120D045B
:10489300E4F00DBD00010CED640A4C70E7B90607A6
:1048A300120B63FF7E0022E964077010120B63751D
:1048B300F00AA4ACF0FDE5662406801BE9640870E9
:1048C30021120B6375F064A4ACF0FDE566240612B7
:1048D3000B67120C552407120B672DFDE43CAF0543
:1048E300FE22E964097033120B63FF7E007C037DB3
:1048F300E8123AA0AC06AD07E5662406120B67750D
:10490300F064120C582407120B67120C552408127A
:0D4913000B672DFDE43CFEAF0522E4FEFF26
:014920002274
:065B48008E658F66A905C1
:105B4E007F057E00120D0FE0C3940A4005120D0F63
:105B5E00E4F00FBF00010EEF64084E70E7E9640732
:105B6E007020E5662405F582E43565F583E075F071
:105B7E000AA4FFE5662406F582E43565F583E02F79
:045B8E00FF227F0073
:015B920022F0
:08339D008E5E8F5F8D608B6175
:1033A500C22AD3E56064809484500302344BE560FF
:1033B5006480948D400302344B120D356003023452
:1033C5004B120C2C123B4433EB0133F60234010350
:1033D500340B04341505341F0634290734330834F7
:1033E5003D0900003447756201756300D22A023435
:1033F50082756201756308D22A023482756201758D
:103405006310D22A8077756201756318D22A806DA0
:10341500756201756320D22A806375620175632820
:10342500D22A8059756201756330D22A804F756240
:1034350001756338D22A8045756201756340D22AC9
:10344500803BC22A8037D3E56064809484402EE5B2
:10345500606480948D5026855F82855E83A3A3E09A
:10346500B4011A855F82855E83A3A3A3E024F67069
:103475000A756201756358D22A8002C22A302A3839
:10348500E4FF120C92E4F00FBF08F7E56024FB851A
:103495006382856283F07F01E55F2404F582E4356C
:1034A5005EF583E5822F120B5BE0FE120C92EEF0C7
:0F34B5000FBF08E4D22B8002C22BAF61126E8AC8
:0134C40022E5
:044729008F5E8D5FB3
:10472D00E55ED3940050030247CCE55E941540033B
:10473D000247CCD22CAF5F1259BD7D5F7F0512664B
:10474D0089AD5EE4FF1266897D527F041266897F12
:10475D00F47E01126C2A75F020E55E900280123B0A
:10476D0038AF828583628F63E0F560603DD394003E
:10477D004046E56094105040E56025E0F5607561B8
:10478D0001E5602401FFE433FEC3E5619FEE648023
:10479D00F87480985022120CF8E0FF120CF8A3E088
:1047AD00FD1265130561056180D77D1B7F061266BD
:1047BD00897D5F7F05126689C22CAF5F0259BDC22C
:0647CD002BAF5F126E8AA3
:0147D30022C3
:10217A008F5E8D5F8B60E55E640A7074E55FC39461
:10218A000A40030222E712231DE4FDFF126689AD0D
:10219A005F1222F6E55F123B4421C20121C80221E7
:1021AA00CE0321D40421DA0521E00621E60721EC39
:1021BA000821F209000021F790052002224190052A
:1021CA002202224190052402224190052602224140
:1021DA0090052802224190052A02224190052C02EC
:1021EA00224190052E022241900530804A0222E0C7
:1021FA00E55E64017052E55FD394004006E55F94A2
:10220A00034006E55F640A703C12231DE55FB40AC9
:10221A000A7D0A1222F6900532801CE55FB4010A93
:10222A007D0B122303900534800DE55FB402137D04
:10223A000C122303900536E0FEA3E0FF126482022B
:10224A0022EE0222E00222E7E55E64026003022235
:10225A00EEE55FD3940050030222E7E55F9407504E
:10226A007CD22CAF601259BD7D277F081266897D0A
:10227A0006E4FF1266897D14E4FF126689E55F248D
:10228A00FE601A14602114602814602F146036242A
:10229A000570437D0112231090053880307D0212AB
:1022AA00231090053980267D0312233390053A8046
:1022BA001C7D0412233390053B80127D05122340B6
:1022CA0090053C80087D0612234090053DE0FF7E84
:1022DA00001264B3800EAF60126BB78007C22BAFD7
:1022EA0060126E8AC22CAF601259BD22E4FF1266D8
:1022FA00897D527F0412668922E4FF1266897D5223
:10230A007F0412668922E4FF1266897D527F0412D5
:10231A00668922D22CAF601259BD7D277F081266CA
:10232A00897D06E4FF12668922E4FF1266897D52DE
:10233A007F0412668922E4FF1266897D527F0412A5
:03234A006689227F
:044AEF008E638F64DF
:104AF3000564E5647002056314F5828E83E0F56650
:104B0300607AC3940850757F2C7E01126C2AE4F5F9
:104B130065E565C395665064856482856383E012A9
:104B23003B444B60004B3E0A4B420B4B480C4B4EF5
:104B33000D4B540E4B5A0F00004B66E4FD802D7D48
:104B43005F7F0780287D5E7F0680227D0A7F02804B
:104B53001C7D327F0280167D467F0280107D0A7F96
:104B630003800A856482856383E0FDE4FF1266891E
:0C4B73000564E56470020563056580952B
:014B7F002213
:061F88008F5E8D5F8B608F
:101F8E00C22AE55E640A600302207CE55F123B44D0
:101F9E001FBD011FD0021FE3031FF60420090520F9
:101FAE001F06203507204B082060090000207812FC
:101FBE0020B17D011220FF756101756200D22A02E7
:101FCE0020981220B17D021220FF75610175620802
:101FDE00D22A0220981220CD7D0312210C756101A8
:101FEE00756210D22A0220981220CD7D0412210C87
:101FFE00756101756218D22A0220981220E9122109
:10200E005F7D0512212F756101756220D22A022093
:10201E00981220E912215F7D0612212F756101753C
:10202E006228D22A0220981221191221737D0712DA
:10203E00213C756101756230D22A02209812211955
:10204E001221737D0812213C756101756238D22A06
:10205E008038122149E4FDFF1266897D091221663E
:10206E00756101756240D22A8020C22A801CE55E0D
:10207E0064017016E55F24F670101221497D0A1274
:10208E002166756101756258D22A302A09AF62AE97
:10209E0061124AEF8005AF60126BB7C22CAF6012AF
:0220AE0059BD1A
:1020B00022D22CAF601259BD7D577F021266897DF6
:1020C00005E4FF126689E4FDFF12668922D22CAF77
:1020D000601259BD7D577F021266897D05E4FF12AB
:1020E0006689E4FDFF12668922D22CAF601259BDC9
:1020F0007D577F021266897D05E4FF12668922E41E
:10210000FF1266897D527F0412668922E4FF1266FF
:10211000897D527F0412668922D22CAF601259BD8C
:102120007D577F021266897D05E4FF12668922E4ED
:10213000FF1266897D527F0412668922E4FF1266CF
:10214000897D527F0412668922D22CAF601259BD5C
:102150007D577F021266897D05E4FF12668922E4BD
:10216000FDFF12668922E4FF1266897D527F041208
:0A217000668922E4FDFF1266892251
:1034C5008F72E572D3945940107D5A1235AC24A6FB
:1034D500FD70030235AB0235A6E572D3944F401655
:1034E500E572945A50107D501235AC24B0FD70032E
:1034F5000235AB0235A6E572D394454016E57294C4
:103505005050107D461235B424BAFD70030235AB18
:103515000235A6E572D3943B4012E5729446500CF1
:103525007D3C1235B424C4FD607C8075E572D3946E
:10353500314012E572943C500C7D321235BC24CEDC
:10354500FD6063805CE572D394274012E572943286
:10355500500C7D281235BC24D8FD604A8043E572A5
:10356500D3941D4016E572942850107D1EE4FF1279
:103575006689E57224E2FD602D8026E572D39413F9
:103585004016E572941E50107D14E4FF126689E51D
:103595007224ECFD60108009E572C394145007ADE8
:1035A50072E4FF12668922E4FF126689E57222E45D
:0F35B500FF126689E57222E4FF126689E5722231
:1059BD008F6AE56A700C302C097F01126EFB7FC077
:1059CD00801FE56A700C202C097F01126EE87FC0E4
:1059DD008026E56AB40112302C0F7F02126EFB7F18
:1059ED0030120016C22E02696CE56AB40114202C27
:1059FD00117F02126EE87F30126EB47FC87E0012E6
:035A0D006C2A22DE
:106948008F69D22C1259BD7D607F021266897D3213
:106958007F061266897D1E7F05126689C22CAF6983
:046968001259BD22E1
:106BB7008F69D22C1259BD7D607F021266897D30A4
:0D6BC7007F03126689C22CAF691259BD22EE
:0E6E8A008F68302B03026948AF68126BB72285
:105D9A00EF24FE60101460162402701C7F01126E3C
:105DAA00FB7F8080107F02126EFB7F2080077F03BB
:105DBA00126EFB7FA01200167FF47E01126C2A7508
:105DCA004204E54270FC7F647E00126C2A7F031253
:085DDA006EE87FA0126EB422F6
:1064B3008E618F627C007D0A123AB2AD07E4FF124F
:1064C30066897D5B7F06126689AE61AF627C007D63
:1064D3000A123AB2E4FF1266897D4A7F070266898F
:046482008E618F6236
:106486007C007D3C123AB21234C57D057F06126649
:1064960089AE61AF627C007D3C123AB2ED4C600C75
:0C64A600AF051234C57D4A7F07126689DD
:0164B20022C7
:025F6D008D5E47
:105F6F00120C0C402FEF648094955028120A8D78F4
:105F7F0005C333CE33CED8F9120D1AFEE4FD0FEF61
:105F8F00AA0670010E14F5828A83E4F00DBD20EE8F
:0B5F9F00D22B8002C22BAF5E126E8A74
:015FAA0022D4
:105FE9008F5E900540E0D394024015D22C1259BD22
:105FF9007542037F327E00126C2AE54270FC8015DF
:10600900D22CAF5E1259BD7D1B7F061266897D0CAD
:0D6019007F03126689C22CAF5E1259BD22B2
:106D8F007E10900540E4F0A3DEFC7E10D22B126E35
:016D9F008A69
:016DA00022D0
:106DA100BF0A02E4FFBD0A02E4FDEF75F00AA42D5B
:026DB100FF22BF
:106C0E00EFD394094002E4FFEDD394094002E4FD72
:0C6C1E007804EF08800123D8FD4DFF2210
:1040960007010203040506070707060504030201D4
:1040A60003010A0A030307050303020503020A0ABA
:1040B60004050A0A0104050A0A0A04050A0A020393
:1040C600070A0A03040A0A04024B00020032072EFA
:1040D60003024B0002003202055F000302055F0087
:1040E6000402055F000502055F000604072E082688
:1040F6000640033204072E08260640025304081E13
:1041060008260452010008024B00020032072E085E
:104116001E08260452010003072B02350636030744
:104126002B0235063803072B0235072603072B0219
:1041360035025302055F000F02055F001002055F9E
:10414600001102055F001202055F001302055F0001
:0A41560014080C0A1D020500241BCA
:105261007461F0A37420F0A37452F0A37401F0A34D
:1052710022A3F0A37461F0A37440F022F0A374039D
:10528100F0E4A3F0A37410F0A37403F0E4A3F0A37B
:10529100227461F0A37441F0A3227461F0A3F0A31E
:1052A1007430F0A3227496F0A37432F0A37495F0D5
:1052B100A3741EF0A322F0A37461F0A314F0A374ED
:1052C10070F0A3E4F022A3F0A37452F0A3223CF502
:0952D10083E0FEEF3395E0FC22BE
:10003E007E407F967C017D507B081260DB7E407F88
:10004E009E7C017D587B081260DB7E407FA67C0182
:10005E007D007B041260DB7E407FB27C017D087BDD
:10006E00041260DB7E407FAE7C017D107B0412604B
:10007E00DB7E407FAA7C017D187B041260DB7E4014
:10008E007FBB7C017D207B051260DB7E407FB67CD2
:10009E00017D287B051260DB7E407FC07C017D30B8
:1000AE007B051260DB7E407FC57C017D387B0412B0
:1000BE0060DB7E407FC97C017D407B041260DB7E6D
:1000CE00407FCD7C027DA07B091260DB7E407FD617
:1000DE007C027DC07B071260DB7E407FDD7C027D73
:1000EE00E07B051260DB7E407FE27C037D007B05BA
:1000FE001260DB7E407FE77C037D207B051260DB98
:10010E007E407FEC7C037D407B051260DB7E407F72
:10011E00F17C037D607B091260DB7E407FFA7C03FD
:10012E007D807B091260DB7E417F037C037DA07B9B
:10013E00091260DB7E417F0C7C037DC07B11126057
:10014E00DB7E417F1D7C037DE07B071260DB7E4101
:10015E007F247C047D007B071260DB7E417F2B7C3D
:10016E00047D207B071260DB7E417F327C047D4064
:10017E007B071260DB7E417F397C047D607B05123C
:10018E0060DB7E417F3E7C047D807B051260DB7EE2
:10019E00417F437C047DA07B051260DB7E417F485E
:1001AE007C047DC07B051260DB7E417F4D7C047D2F
:1001BE00E07B051260DB7E417F527C057D007B0576
:1001CE001260DB7E417F577C057D407B091260DB30
:1001DE009000297417F07F031263EA9000287419B7
:1001EE00F090002074B1F09000217491F0900022F4
:1001FE007403F0900023747FF090002404F09000BC
:10020E00257403F0E4900026F0900027F090003063
:10021E00740912527D7415F0A37403F0A3741512B1
:10022E00527D7409F0A37403F0E4FFEFFD3395E003
:10023E00FC74302DF58274001252CF74102DF5829D
:10024E0074003CF583EEF00FBF08E0E4FFEFFD33E2
:10025E0095E0FC74382DF58274001252CF74182D6F
:10026E00F58274003CF583EEF00FBF08E090052098
:10027E00E4F0A374B4F0900522E4F0A374B4F0900B
:10028E0005247401F0A374E0F0900526E4F0A37445
:10029E0078F09005287402F0A37458F090052AE4C3
:1002AE00F0A3743CF090052C7402F0A37458F07413
:1002BE000790052EF0A3F0900530F0A3F0900532D4
:1002CE00F0A3F0900534F0A3F0900536E4F0A3749B
:1002DE003CF0900538740AF09005397428F09005BA
:1002EE003A7405F090053B740AF090053CF09005C9
:1002FE003D7428F09000A47401F0900B607415F01A
:10030E00A37411F09000A57401F0900B807415F099
:10031E00A37410F09000A67401F0900BA07415F069
:10032E00A37421F09000A77401F0900BC07415F027
:10033E00A37420F09000A87401F0900BE07415F0F7
:10034E00A37431F09000A97401F0900C007415F0B4
:10035E00A37430F09000AA7401F0900C207415F084
:10036E00A37441F09000AB7401F0900C407415F042
:10037E00A37440F09000AC7401F0900C60745312B2
:10038E00526B743612526B7438F0A3E4F0A37453AC
:10039E00F0A3E4F09000AD04F0900C807453125270
:1003AE006B7434F0A37421F0A37453F0A3E4F090B3
:1003BE0000AF04F0900CC01252697430F074031246
:1003CE0052C7E4F09000B004F0900CE01252697441
:1003DE0030F074041252C7E4F09000B104F0900DA6
:1003EE0000125261743212526B7452F0A37420F0E8
:1003FE009000B27401F0900D201252617432F0A38D
:10040E0074021252C87420F09000B37401F0900D73
:10041E0040745312526B7433F0A3E4F09000B404A2
:10042E00F0900D601252927430F07402125272906B
:10043E0000B57401F0900D801252927430F0740574
:10044E001252729000B67401F0900DA01252927476
:10045E0030F0A374061252739000B77401F0900D31
:10046E00C01252921252A67498F0A3744B12527389
:10047E009000B87401F0900DE01252921252A674D0
:10048E0093F0A374181252739000B97401F0900E89
:10049E00001252927430F0A37413125273A374703C
:1004AE00F0A37402F09000BA14F0900E2012529B3A
:1004BE007412F0A3747012526B7461F0A314F09066
:1004CE0000BB7401F0900E4012529B74111252B781
:1004DE009000BC04F07461900E6012529D74141260
:1004EE0052B79000D104F09011001252927492F013
:1004FE00A3744BF0A37490F0A37402F0A37490F065
:10050E00A37432F07499A3F0A3F0A3746012526B2B
:10051E00749112526B7491F0A3E412527390000F07
:10052E007401F0125DE27F01126EFB7F4012001625
:10053E007D2F7F071266897D0C7F031266897D32BF
:0C054E007F061266897D1E7F05126689FB
:01055A00227E
:0A60DB008E5A8F5B8C5C8D5D8B5E2E
:1060E500E4F9C3E55E6480F8E96480985022E9FF2D
:1060F5003395E0FEE55B2FF582E55A3EF583E493A3
:10610500FDE55D2FF582E55C3EF583EDF00980D276
:016115002267
:10556F00AF6AEF3395E0FEE56975F008A42428F5DE
:10557F0082E43400F583E5822FF582E5833EF583DF
:10558F00E0FFE56AFD3395E0FC22AB66AD65AF64E5
:10559F00223EF583E0FD74B82FF582741D3EF5832E
:1055AF00EDF0056AE56A22EF3395E0FEEF25E0FFA7
:1055BF00EE33FE22A2E0CE13CE13223CF583EFF0A2
:0555CF00056AE56A22F7
:045B93008C5B8D5C3E
:105B9700EF6043D201D202D20CE4F55D855C8285C9
:105BA7005B83E0FEA3E04E6027AF5D1255B6E55C70
:105BB7002FF582E55B3EF583E0FEA3E0FF12445933
:105BC700922820280B055DC3E55D6480949040CC46
:065BD700C201C202C20C73
:015BDD0022A5
:045BDE008C608D61E9
:105BE200EF6043D201D202D20CE4F5628561828574
:105BF2006083E0FEA3E04E6027AF621255B6E56116
:105C02002FF582E5603EF583E0FEA3E0FF124459E2
:105C1200922C202C0B0562C3E5626480949040CCE8
:065C2200C201C202C20C27
:015C28002259
:04445900AD07AC06F9
:10445D00C22D780CEF0880031255C3D8FB540FF50D
:10446D00637808AF05AE04EF0880031255C3D8FB7F
:10447D00540FF5647804AF05AE04EF0880031255B0
:10448D00C3D8FB540FF565ED540FF566E563607108
:10449D00B40108125599123C4D8066E563B40208CB
:1044AD00125599126B228059E563B4030812559980
:1044BD00123990804CE563B40408125599126AC301
:1044CD00803FE563B405081255991224FD8032E54D
:1044DD0063B4060812559912127D8025E563B40761
:1044ED0008125599125AFC8018E563B40808125544
:1044FD009912574E800BE563B4090612559912684F
:03450D00B5A22D27
:014510002288
:103C4D008F678D688B69E567B40113900020E0FFE5
:103C5D001258B7900020EFF0FD7F20023D0AE56776
:103C6D00B40211900021123D10900021EFF0FD7F64
:103C7D0021023D0AE567B40311900022123D109018
:103C8D000022EFF0FD7F22023D0AE567B40410909B
:103C9D000023123D1A900023EFF0FD7F23805EE597
:103CAD0067B40516900024123D1A900024EFF0FD24
:103CBD007F247E0012637F0264E3E567B4061090F3
:103CCD000025123D24900025EFF0FD7F25802EE587
:103CDD0067B40710900026123D24900026EFF0FDEA
:103CED007F268019E567B40819900027E0FFAB69BE
:103CFD00AD681258B7900027EFF0FD7F277E0012B8
:103D0D00637F22E0FFAB69AD681258B722E0FFABCD
:103D1D0069AD681258B722E0FFAB69AD681258B7AC
:013D2D002273
:1058B700D22EAC07BD01047E018033BD02047E02F7
:1058C700802CBD03047E048025BD04047E08801E51
:1058D700BD05047E108017BD06047E208010BD071D
:1058E700047E408009BD08047E808002C22EBB0171
:1058F70005EE4204800BEB7006EEF452048002C200
:075907002E302E03AF042235
:01590E002276
:026B22008B677F
:106B2400C22EEF7016ED7013E5677003025C74E516
:0B6B340067B401077880E6FF125A608A
:016B3F002233
:063990008F678D688B6952
:10399600E5677007123A76E4FD801AE567B4010719
:1039A600123A767D01800EE567B4020CAD69AF6808
:1039B600126E987D02024F5EE567B40306124D2F24
:1039C600C21D22E567B40415AD69AF6812641E8F87
:1039D60043754205E5427003023A7580F7E5676470
:1039E600067017E5687013F56A12556F74102DF599
:1039F6008274001255CAB408F022E567640770178E
:103A0600E5687013F56A12556F74182DF582740007
:103A16001255CAB408F022E56764087027E5687095
:103A260023E569701FF56AAF6AEF3395E0FE7410FF
:103A36002FF58274001255A0B408EC754201E542D8
:103A4600602D80FAE56764097025E5687021E569EF
:103A5600701DF56AAF6AEF3395E0FE74182FF58294
:0F3A660074001255A0B408EC754201E54270FCE3
:093A750022AD69AF68126E9822BF
:106AC3008F67AE03AF05E567D394004012E5679483
:106AD30007500CAD06126E98AD07AF671266DD2244
:1024FD008F678D688B69E5677018E5687014E569FD
:10250D0070057F01126EB4E569640160030226AAAD
:10251D008043E567701CE568B40117E56970057FB8
:10252D0004126EB4E569640160030226AA7F0402F9
:10253D0026A7E5677029E56864027023E5697005D3
:10254D007F05126EB4E569640160030226AA90004E
:10255D000FE0B403057F010226A77F050226A7E53C
:10256D0067B4011BE5687017E56970057F02126E8F
:10257D00B4E569640160030226AA7F020226A7E57D
:10258D0067B4011CE568B40117E56970057F081291
:10259D006EB4E569640160030226AA7F080226A7CE
:1025AD00E56764017029E56864027023E5697005CB
:1025BD007F0A126EB4E569640160030226AA9000D9
:1025CD000FE0B403057F020226A77F0A0226A7E5C6
:1025DD0067B4021BE5687017E56970057F40126EE0
:1025ED00B4E569640160030226AA7F400226A7E5CF
:1025FD0067B4021CE568B40117E56970057F101218
:10260D006EB4E569640160030226AA7F100226A755
:10261D00E56764027024E5686402701EE569700563
:10262D007F50126EB4E5696401707290000FE0B4D2
:10263D0003047F4080647F508060E567B40317E535
:10264D00687013E56970057F80126EB4E5696401E9
:10265D00704B7F808044E567B40318E568B40113BF
:10266D00E56970057F20126EB4E5696401702E7FF7
:10267D00208027E56764037024E5686402701EE519
:10268D006970057FA0126EB4E569B4011090000F5A
:0E269D00E0B403047F8080027FA012001622AA
:10127D008F678D688B69E5677017AD69AF68126E02
:10128D00988E348F35D3E5359400E534940050F5C0
:10129D0022E567B4011BE568B40116E5697007C264
:1012AD002F7F0112300AE569640160030214EA80A0
:1012BD0058E5676401702BE56864027025E5697077
:1012CD0007C22F7F0212300AE56964016003021420
:1012DD00EA90000FE0640370030214EAD22F7F023C
:1012ED008031E5676401702EE56864037028E56957
:1012FD007007C22F7F0312300AE569640160030293
:10130D0014EA90000FE0B40306D22F7F018004D2BF
:10131D002F7F0302300AE5676401702DE5686404D0
:10132D007027E569700CC22F7F0112300A7F4012C1
:10133D006EB4E569640160030214EAD22F7F0112D5
:10134D00300A7F40120016807CE5676401703AE533
:10135D006864057034E569700CC22F7F0212300A83
:10136D007F10126EB4E569640160030214EA900007
:10137D000FE0640370030214EAD22F7F0212300AC9
:10138D007F10120016D22E803EE5676401703BE59A
:10139D006864067035E569700CC22F7F0312300A40
:1013AD007F50126EB4E569640160030214EAD22F16
:1013BD007F0312300A90000FE0B403047F408002D7
:1013CD007F50120016C22E02696CE5676402702907
:1013DD00E56864017023E56970057F100214D1E59D
:1013ED0069B401057F100214DBE569640260030234
:1013FD0014EAD22E7F010214E7E56764027029E535
:10140D006864027023E56970057F200214D1E569D7
:10141D00B401057F200214DBE56964026003021448
:10142D00EAD22E7F020214E7E56764027029E568AF
:10143D0064037023E56970057F400214D1E569B43A
:10144D0001057F400214DBE569640260030214EAC2
:10145D00D22E7F030214E7E56764027023E568640A
:10146D0004701DE56970047F808059E569B401043D
:10147D007F80805AE56964027063D22E7F04805AA2
:10148D00E56764027023E5686405701DE569700405
:10149D007F048030E569B401047F048031E569641F
:1014AD0002703AD22E7F058031E5676402702EE519
:1014BD0068640670287D017F07124ED6401FE569CE
:1014CD0070057F08026EE8E569B401057F08026EBC
:0E14DD00FBE569B40207D22E7F061229952284
:025AFC008B67B6
:105AFE00EF7037ED7034E567700690000F0480206C
:105B0E00E567B4010A90000F7402F0D22E801BE5F7
:105B1E0067B40216C21D7FFF126EB490000F74039D
:105B2E00F0C22F7F0212300AD22E302E0C90000FB0
:095B3E00E0FD7F0F7E0012637F81
:015B4700223B
:10574E008F678D688B69E567700C125792749F2F67
:10575E00F58274008019E567B4010C125792749F9C
:10576E002FF58274008016E567B4020912579A3E2F
:10577E00F583E4F022E567B4030912579A3EF583E8
:10578E007401F022AD69AF68126E9822AD69AF68F0
:0B579E00126E98746F2FF582740022C9
:0268B5008F67EB
:1068B700AF057804EF08800123D8FD4BF568E5673D
:1068C700B40908E568B499030253C4AD68AF671209
:0268D700651347
:0168D900229C
:0D6E9800EF75F00AA47C002DFFEC35F0FE34
:016EA50022CA
:0466DD008F688D69CC
:1066E100C3E569648094E4501BE4F56AC3E5696419
:1066F10080F8E56A648098500BC22EAF6812299524
:04670100056A80E8BD
:016705002271
:0D6EA600C296007F0512681F126450D2963C
:016EB30022BC
:106D2700126EA6EF20E0F9C296007F0612681FC216
:066D3700B60000D2962216
:106D3D00126EA6EF20E0F9C296007F0412681FC202
:066D4D00B60000D2962200
:045FAB008E608F6114
:105FAF00AE04AF058E638F64C296007F0312681F25
:105FBF00E560FF12681FAF6112681FE4F56212649B
:105FCF0050E5642562F582E43563F583EFF00562F1
:095FDF00E562C3942040E7D2966C
:015FE8002296
:085C29008E658F668C678D68A3
:105C3100126EA6EF20E0F985656A85666BC2960053
:105C41007F0212681FE567FF12681FAF6812681FA5
:105C5100E4F569E56B2569F582E4356AF583E0FFD2
:105C610012681F0569E569C3942040E7C2B60000C8
:025C7100D296C9
:015C7300220E
:0A5509008E5A8F5B8C5C8D5D8B5E0B
:10551300C2AF126D27126EA6EF20E0F9855C60859D
:105523005D61C296007F0212681FE55AFF12681F71
:10553300AF5B12681FE4F55FAF5EEF3395E0FEC328
:10554300E55F9FEE6480F87480985014E561255FF1
:10555300F582E43560F583E0FF12681F055F80D8AC
:0B556300C2B60000D296126D3DD2AF20
:01556E00221A
:10637F008E718F728D73C2AF126D27126EA6EF20C2
:10638F00E0F9C296007F0212681FE571FF12681FC5
:10639F00AF7212681FAF7312681FC2B60000D29699
:0663AF00126D3DD2AF2289
:10606300C2AFE4F55BF55CF55DF55EF55FF55AAE41
:106073005EAF5FAC5BAD5C125FAB7420255CF55C1F
:10608300E4355BF55B7420255FF55FE4355EF55E13
:0B609300055AE55AC3948940D6D2AFED
:01609E0022DF
:105DE200C2AF756200756300756400E4F560F56129
:105DF200F55F126D27AE63AF64AC60AD61125C29D2
:105E020074202561F561E43560F56074202564F540
:105E120064E43563F563055FE55FC3948940D3129B
:045E22006D3DD2AF51
:015E26002259
:105636000500050105030507050F051F051E051CC9
:10564600051805100201040E040A03060101040BE5
:105656000304040F020304010302040D0200020204
:1056660003000409040403050307010003030407F8
:10567600030104060402040C0516051500000615B0
:0E568600062A060C06380633061E0612061704
:104CA0002430F58274003EF583EDFF3395E0FEE598
:104CB000822FF582E5833EF583E0FFEDFB3395E03F
:104CC000FA22AF4112681FC293126EF2D293D2AF92
:104CD000223EF583E0FC74B82FF582741D3EF58307
:104CE000ECF00D221528E528D394002225E0243687
:104CF000F582E43456F583E49322E4F57CD20EC2C7
:104D000026C21CC219227FA0126EB4E4F542C21D55
:104D100022126EF2D2B67801EF0822122C47D2CAC4
:0F4D2000D20ED22622ECFF3395E0FEEF7803226D
:10416000200E2F900540E004F577D36480948150B1
:1041700003024220D3E5776480948F400375770F64
:10418000900029E0FF122C4790002AE0F576124CAF
:10419000FA22301958302612124CE4400302422011
:1041A000C2CAC226D21C85762822301C0A124CE4D0
:1041B000506EC226C21C22AF7A157AEF700BC2195C
:1041C000E57625E0F528D21C22E57B30E0058576F2
:1041D000288008E57675F003A4F528AF7B7801EF19
:1041E00008800103D8FDF57BD226D2CA22D57708F4
:1041F000C20EE4F542C21D22057C7440257CF58286
:10420000E43405F583E0124CEC540FF57A74019315
:10421000F57B700AD21CE57625E025E0F528D21959
:01422000227B
:1050EF00200E12900029E0FF122C4790002AE0F5C5
:1050FF0078124CFA2230195130260F124CE4505DC1
:10510F00C2CAC226D21C85782822301C0A124CE44F
:10511F00504BC226C21C22AF7A157AEF7007C21904
:10512F00C20EF54222E57B30E0058578288008E540
:10513F007875F003A4F528AF7B7801EF08800103A1
:10514F00D8FDF57BD226D2CA22E543124CECFA7475
:0D515F000193FBEA540FF57AEBF57BD219B2
:01516C002220
:10645000E4F575D297F574C2B6126EF2AF75780195
:10646000EF08800123D8FDF57530970343750112BD
:106470006EF2D2B60574C3E5746480948840D8AFD8
:0164800075A6
:0164810022F8
:096EF20000000000000000002275
:10665D00C2B7E4FEC2B6126EF2EF30E704D2B580D7
:10666D0002C2B5124D11800123D8FDFF126EF20E3C
:0B667D00BE08E1C2B6D2B7D2B6D2B55B
:0166880022EF
:0D001600C2AFEF4227AF2712665DD2AF22C6
:0E6EB400C2AFEFF45227AF2712665DD2AF22B5
:10681F00E4FEC2B6126EF2EF30E704D2B58002C2C8
:10682F00B5124D11800123D8FDFF126EF20EBE0876
:05683F00E1D2B6D2B564
:016844002231
:096EFB00C2AFEF4241124CC22269
:0A6EE800C2AFEFF45241124CC22277
:102C4700EF123B442CAF012CB6022CBD032CC4045D
:102C57002CCB052CD2062CD9072CE0082CE7092C05
:102C6700EE0A2CF50B2CFC0C2D030D2D0A0E2D1145
:102C77000F2D18102D1F112D26122D2D132D341445
:102C87002D3B152D42162D49172D50182D57192D4F
:102C97005E1A2D651B2D6C1C2D6E1D2D751E2D7C32
:102CA7001F2D832000002D6C75CB8E75CAC622752B
:102CB700CB9575CA772275CB9B75CA692275CBA050
:102CC70075CABA2275CBA675CA332275CBAB75CA3E
:102CD700632275CBB075CA022275CBB475CAA3221D
:102CE70075CBB875CAFA2275CBBC75CAD82275CB15
:102CF700C075CAA82275CBC475CA362275CBC775ED
:102D0700CA862275CBCA75CABC2275CBCD75CAB423
:102D17002275CBD075CA762275CBD375CA3022758A
:102D2700CBD575CAB22275CBD875CA132275CBDA43
:102D370075CA522275CBDC75CA7D2275CBDD75CA83
:102D47006E2275CBE075CA542275CBE275CA1B2279
:102D570075CBE375CAC32275CBE575CA5E2275CB01
:102D6700E675CADA22801C75CBE875CA902275CB46
:102D7700EA75CAD92275CBEC75CA092275CBED75F0
:0A2D8700CA292275CBE875CA412263
:10002600C3EF648094A15008EF25E025E0F528226F
:04003600E4F52822A3
:0235C4008F5A1C
:1035C600900118E0FFE55A7006E545D39F5012E5D5
:1035D6005A640160030236BAE546D39F50030236A9
:1035E600BAE55A7018C3E5459FF55D74602FF582FC
:1035F600E4341EAD82F55E8D5F7F40801BE55AB4D4
:103606000119C3E5469FF55D74B02FF582E4341EBB
:10361600AF82F55E8F5F7F101200167FF47E011277
:103626006C2A7D207F051266897D1A7F08126689BD
:103636007FC87E00126C2AE4F55BE55BC3955D509E
:1036460061055FE55FAE5E7002055E14F5828E83EE
:10365600E0F55C123B4436970036750A36790B3630
:103666007F0C36850D368B0E36910F0000369DE4A5
:10367600FD80277D5F7F0780227D5E7F06801C7D23
:103686000A7F0280167D327F0280107D467F02808F
:103696000A7D0A7F038004AD5CE4FF126689055B40
:1036A6008098E55A70047F408007E55AB401057F8B
:0436B60010126EB4CC
:0136BA0022ED
:10506C00200E10754406901DB8E06003D20E22E4A9
:10507C00F54222E528D394004003152822C2CA1514
:10508C0044E54414603D14603214601D1460151422
:10509C007049901DB8E0FF7003F54222122C479026
:1050AC001DB9802F901DBA8015901DBBE0FF7003B9
:1050BC00F54222122C47901DBC8018901DBDE0FFBC
:1050CC00020026901DBEE0FF7003F54222122C4711
:1050DC00901DBFE0FF120026D2CA22E4F542C2CADC
:0350EC00C20E22CF
:10660100900028E0FF6026200E07124D1B7528140C
:1066110022E528D394004003152822202608D2CA57
:0E662100752814D22622C2CA75287DC22622F0
:1065A300200E0C7F1C124D1B75286475793C22E567
:1065B30028D394004003152822AF791579D3EF64CB
:0E65C300809480400475286422C20EE4F542E4
:0165D10022A7
:1062A600E54214601C14601C14601F146022146004
:1062B6002224057021C2CAC20EC226C21CE4F544BD
:1062C6002202506C126601D21D22124160D21D229A
:0762D6000265A31250EF2244
:1063EA00BF010790002A7418F022BF020790002A02
:1063FA007412F022BF030590002A8014BF0407908C
:10640A00002A740BF02290002ABF05047409F022B6
:04641A00740CF022EC
:024FE600AC0716
:104FE800C3EC64809480404AEC64809488504320E9
:104FF8002A21E4FD124D25C333CE33CED8F9124C05
:10500800A074102BF58274003AF583EFF00DBD08FB
:10501800E3801FE4FD124D25C333CE33CED8F912F9
:105028004CA074182BF58274003AF583EFF00DBD8F
:1050380008E3202A16E4FDEDFF3395E0FE74102FF7
:10504800F5827400124CD1BD08ED22302A15E4FD1A
:10505800EDFF3395E0FE74182FF5827400124CD1E1
:03506800BD08ED93
:01506B002222
:1053C4007D3F7F091266897D507F08126689906F40
:1053D4002412542B7D5B7F06126689906F2512542C
:1053E4002B906F26E493FDE4FF126689906F27E407
:1053F4009324BE601414601514601814601B1460A8
:105404001E240570217D0A80067D3280027D467F40
:105414000280107D0A7F03800A7D287F0380047D3B
:10542400467F0312668922E493FDE4FF1266892213
:105EED008F5BE55B7005D22CFF8009E55BB4010784
:105EFD00D22C7F011259BD7D4B7F021266897D0226
:105F0D00E4FF1266897D32E4FF1266891253C4E5FF
:105F1D005B70028005E55BB401057F40126EB42213
:103D2E00A209300501B350307D017F04124ED650EA
:103D3E002320050E30090B9000A4E0FF7C0B7D6064
:103D4E00800F30050F20090C9000A5E0FF7C0B7D45
:103D5E0080125BDEA2099205A20A300601B3503032
:103D6E007D027F04124ED6502320060E300A0B9091
:103D7E0000A6E0FF7C0B7DA0800F30060F200A0C02
:103D8E009000A7E0FF7C0B7DC0125BDEA20A9206BC
:103D9E00A20B300701B350307D037F04124ED65074
:103DAE002320070E300B0B9000A8E0FF7C0B7DE06C
:103DBE00800F30070F200B0C9000A9E0FF7C0C7DCC
:103DCE0000125BDEA20B9207A20D300801B3503039
:103DDE007D047F04124ED6502320080E300D0B901A
:103DEE0000AAE0FF7C0C7D20800F30080F200D0C08
:103DFE009000ABE0FF7C0C7D40125BDEA20D9208C2
:013E0E002291
:1064E300534103900024E0FE543FFF7804088001E9
:1064F30023D8FD54F0FFEE30E40343070490002457
:0F650300E030E503430708EF4241C2AF124CC23C
:016512002266
:022995008F6B46
:10299700302E05756CF48003756C64E56B6401700B
:1029A70029AF417803EF08800123D8FD33922F7FA9
:1029B70010202F0B122AB17F10126EE8022AA912DB
:1029C7002ABC7F10126EFB022AA9E56B64027028ED
:1029D700AF417802EF08800123D8FD33922F7F2083
:1029E700202F0A122AB17F20126EE88008122ABC13
:1029F7007F20126EFB022AA9E56B64037028AF41A2
:102A07007801EF08800123D8FD33922F7F40202FD4
:102A17000A122AC77F40126EE88008122AD27F4026
:102A2700126EFB022AA9E56B6404701EE54133921E
:102A37002F7F80202F0A122AC77F80126EE8800816
:102A4700122AD27F80126EFB8058E56B64057027CF
:102A5700AF417805EF08800123D8FD33922F7F041B
:102A6700202F0A122ADD7F04126EE88008122AE856
:102A77007F04126EFB802BE56B6406702CAF4178E8
:102A870004EF08800123D8FD33922F7F08202F0AF7
:102A9700122ADD7F08126EE88008122AE87F0812E2
:092AA7006EFBAF6C7E00126C2A7C
:102AB00022126EFBAF6C7E00126C2A22126EE8AFFF
:102AC0006C7E00126C2A22126EFBAF6C7E00126CC0
:102AD0002A22126EE8AF6C7E00126C2A22126EFB64
:102AE000AF6C7E00126C2A22126EE8AF6C7E001270
:032AF0006C2A222B
:105D5100900024E030E0057F10126EFB900024E0FB
:105D610030E1057F20126EFB900024E030E2057FD8
:105D710040126EFB900024E030E3057F80126EFB41
:105D8100900024E030E4057F04126EFB900024E0D3
:095D910030E5057F08126EFB22CB
:106C7B0030030A124D06C203C210C21D2230040992
:0A6C8B00124D06C204C212C21D22FF
:106513008F708D71E570B4011FE5717003125C74A7
:10652300E571B401077880E6FF125A60E571B43271
:106533000E7FF47E01026C2AAD71AF701266892260
:10668900EFFEEDFF1280008E2D8F2E12534F757481
:1066990032AF741574EFD39400400EE4F573E573CB
:0966A900C3943A50EC057380F52E
:0166B20022C5
:10534F00D2A8AFA875A881C213852E82852D83E4BC
:10535F0093C4540FFE4306F08E80C284D28500C2E0
:10536F00870000D287007580FF7580FEC284C285DA
:10537F0000C2870000D287007580FFD2137D407C6A
:10538F001FE4FE30B40D0EBE32F9ED1D70011CEDA1
:10539F004C70EE7C1F7D40E4FE20B40D0EBE32F942
:1053AF00ED1D70011CED4C70EE8FA8C2A87F0A7E18
:0453BF0000126C2A42
:0153C30022C7
:1066B3007580FDC284C28500C28700000000D287B6
:1066C300007580FF7F0A7E00126C2A7F997E091273
:0A66D30080008E2D8F2E12534F22EF
:10422100D284D285C286A2809216A281921FA282D6
:104231009217A2839220D2862001537D027F011220
:104241004ED640137D037F01124ED6400A30160729
:10425100301832D22380377D027F01124ED6500FA3
:1042610030160C301F09301804D223802180167DAE
:10427100037F01124ED65012201603301F0C301846
:1042810004D22380091267808004C218C22320024D
:104291004E7D027F02124ED640127D037F02124EE6
:1042A100D64009301706301A2FD224227D027F0210
:1042B100124ED6500E30170B302008301A03D2247C
:1042C1002280157D037F02124ED6500F2017033036
:1042D1002009301A03D224220267A8C21AC224225A
:10678000753D1E753E60E4FFE53E2FF582E4353D24
:10679000F583E4F00FBF50F0753D1E753E60E4F5E3
:0767A00045C225C210D2180A
:0167A70022CF
:1067A800753F1E7540B0E4FFE5402FF582E4353FA4
:1067B800F583E4F00FBF10F0753F1E7540B0E4F5A7
:0767C80046C227C212D21ADB
:0167CF0022A7
:106BD400C284D285C286A2809209A281920AA2822C
:0D6BE400920BA283920DD286D284D285221C
:10611600E57E2560F582E4357DF5832274FF123B2A
:106126001AE4FBFAF9F8C3023B07057F7480257E63
:10613600F57EE4357DF57D22F582E4341DF5832276
:0B614600757F01757D00757E20E4224E
:1042E1007D027F07124ED650057F04126EE8C22868
:1042F100D222E4F5427FE87E03126C2AC298C2AF53
:10430100C22F7F0312300A755E7F755D96755C98CA
:10431100755B00785B126122504430983E120006B2
:10432100126E0BEF14601824F0602624C1600B2478
:10433100F670287F06126F0D80211261C6801C7FE6
:1043410006126F0D1269B21264E3125DE2D2288087
:104351000A7F06126F0D125A10D2283028B5E47860
:1043610085F6D22F7F0112300A7F40120016C22E2D
:1043710012696C7D467F021266897D1E7F07126677
:10438100897D147F081266897D327F03126689C296
:0D4391002F7F0312300A7FFF126EB4C2228C
:01439E0022FC
:105A1000126146F55F7F02126F0DE57F2402F5618A
:105A2000AF7F126F0DE4F560126116E0FF126F0D8B
:105A3000126116E02561F5610560E560C394804060
:105A4000E7AF61126F0D7F03126F0D126F15EF64D8
:0F5A500015600C126130055FE55FC3942240B60C
:015A5F002224
:1069B200126146F55F12670650077F06126F0D805F
:1069C200057F15026F0D126130055FE55FC39422EA
:0269D20040E3A0
:0169D40022A0
:10670600E4F560126F1574D0256012613EEFF00556
:1067160060E560C3948440EB126DE9901E52E0B5CB
:086726000705126C45D322C3E4
:01672E002248
:106C4500E4FF74D22FF582E4341DF583E0FEE57E82
:0A6C55002F12611AEEF00FBF7FE866
:016C5F002212
:106DE900E4FFFE74D02E12613EE02FFF0EBE82F347
:016DF9002277
:1061C600E4F55FF5657564E0756393756204F561E2
:1061D600786112612250213098F61200068F60E530
:1061E6006064046013AF65056574D02F12613EE5E7
:0861F60060F0255FF55F80D821
:0161FE00227E
:04000600AF99C29854
:01000A0022D3
:086F0D003099FDC2998F992211
:076F15003098FDAF99C2980E
:016F1C002252
:106CE1000C0102030405060708090A0B0C01020343
:086CF1000405060708090A0B5F
:10672F00AF5FEF3395E0FE75F007EF123B38EE7574
:10673F00F007A42583F583E0227883E6FF126CAF80
:09674F00EF22C295D297D2AF22CD
:10684500C22BC2AF126F1D7F83126CF9126AE3125D
:1068550067517884E66F600B125E6A302A05125F15
:056865002D922BA22B77
:01686A00220B
:105F2D007984E778876660367884E6FF7887F6EFC0
:105F3D007013E552C3940A500C7D077F04124ED6A0
:105F4D005003125E277D057F04124ED65010E54199
:105F5D0054036005123FC3D322123FC3C322C32291
:103FC300E4F55F900A5012672F7003024087900A4E
:103FD3005112673660167881666003024087900A43
:103FE3005212672F7888666003024087AF5FEF3312
:103FF30095E0FE900A53126736FF7880E6FEEF6E77
:104003006020EF601DB4080BEED394014005EE94DD
:1040130007400FEF6409706CEE64016005EE6407FE
:104023007062AF5FEF3395E0FE900A54126736FF7C
:10403300F46006EF788366704BE55FFD3395E0FC33
:10404300900A5575F007ED123B38EC12673E788401
:10405300667031D201D20274BD2DF58274003CF535
:1040630083E0FFC007EDAE047805C333CE33CED86B
:10407300F92480F582740E3EAD82FCD007125BDE1C
:10408300C201C202055FC3E55F64809493500302DB
:024093003FC626
:014095002208
:105E27007D087F04124ED6500D7883E6FF126CAFC3
:105E3700EFC39407402CD22F7F0112300A7F401204
:105E47000016C22E12696CD201D202E4FD7F0A123B
:105E57004F5EC201C2027F50126EB4C22F7F011281
:035E6700300A22DC
:105E6A00C2AF126F1D7FBF126CF9126AE37884A663
:105E7A0007126AE37884A607126AE37883A60712F0
:105E8A006AE37888A607126AE37881A607126AE3AA
:105E9A007880A607126AE37882A607126F1D126736
:025EAA00512283
:1057A900C2AF126F1D7F8E1257F87F90126CF97F6E
:1057B900A7126CF9126F1D7FBE126CF9E4FF126C0F
:1057C900F97884E6FF126CF97883E6FF126CF978B0
:1057D90088E6FF126CF97881E6FF126CF97880E6A9
:1057E900FF126CF97882E6FF1257F81267512212FC
:0B57F9006CF9E4FF126CF9126F1D2226
:105A60008F72E572B401047D63803EE572B4020674
:105A70007D087F068035E572B403067D317F08809E
:105A80002AE572B404067D617F08801FE572B405C3
:105A9000067D257F088014E572B406067D597F03D4
:0F5AA0008009E572B407077D487F0712668922E7
:026CAF00AE072E
:106CB100EE54F0FF780408800103D8FD75F00AA4B2
:066CC100FFEE540F2FFF4F
:016CC70022AA
:105C7400126748906CE193FF1234C5788412674A26
:105C8400601B788412674AC3940A50077D327F06EA
:105C94001266897884E6FF126CAF1234C512674825
:105CA400C3940C50067D0A7F0280047D507F061247
:0A5CB40066897D507F051266892283
:105967007FF47E01126C2A7D097F06126689788191
:105977001259AD7D0E7F031266897D357F0612664B
:10598700897D097F0612668978881259AD7D1E7F49
:10599700091266897D1E7F071266897882E6FF12E3
:1059A7006CAF1234C522E6FF126CAF1234C57FF418
:0659B7007E01126C2A22A1
:076F1D00C2B6C295D2952215
:106CF900E4FEC297EF30E002D297C2B6D2B6EFC334
:066D090013FF0EBE08ECB2
:016D0F002261
:106AE300E4FFD297FED2B6C2B6A297E433C43333DF
:0F6AF300335480FDEFC313FFED42070EBE08E6DC
:016B02002270
:1056F100EF3395E0FE74702FF58274003EF583E080
:10570100FF22AF5AEF3395E0FEEF222460F5827459
:10571100013EAD82FCD22822900520E0F547A3E0AE
:10572100F548222450F58274053EAD82FC2290009A
:10573100BAE0FF7C0E7D2022D221D201E4FF22C2F9
:0D57410001C2217F1922D221D22F7F022226
:10283400E5527008126CC88F5202292FE552B40574
:102844000812467C8F5202292FE552B40B08126DF0
:10285400538F5202292FE552B40A08125CBE8F52DC
:1028640002292FE552B40F081260268F5202292F35
:10287400E552B4140812234D8F5202292FE552B4A5
:102884001908126B408F5202292FE552B41E081208
:102894006A1B8F5202292FE552B42308126A818FD2
:1028A4005202292FE552B42807126EC28F52807B40
:1028B400E552B42D071267F88F52806FE552B43297
:1028C400071261FF8F528063E552B43E07126B5EBC
:1028D4008F528057E552B43C07126DB38F52804B30
:1028E400E552B43307126A5F8F52803FE552B44118
:1028F40007126E3C8F528033E552B44C07126E4C73
:102904008F528027E552B44407126E5C8F52801BAD
:10291400E552B4370712585E8F52800FE552B4392E
:10292400071258048F528003E4F552E553700612DF
:10293400000E8F5322E553B40506126F048F532201
:10294400E553B40A06126E6C8F5322E553B40F0696
:10295400126E7B8F5322E553B41406123B6A8F53D5
:1029640022E553B43D06126B7C8F5322E553B43FEA
:10297400061265438F5322E553B443061267D08F82
:102984005322E553B44D06126AA28F5322E4F55341
:012994002220
:106CC8007D077F05124ED6500D30000A90052AE048
:096CD800F52BA3E0F52C7F052249
:10467C00302314200F11C21B7D047F01124ED65023
:10468C00037F0B227F0A227F081262DD500612453F
:10469C00C77F0022202308300F05C20F7F05227D23
:1046AC00057F06124ED6501EE5394538701890001D
:1046BC00B5E0FF7C0D7D80125BDE90052EE0F538B9
:1046CC00A3E0F53980487D067F06124ED6501EE5D4
:1046DC003C453B70189000B6E0FF7C0D7DA0125B52
:1046EC00DE900530E0F53BA3E0F53C80217D077FB3
:1046FC0005124ED6500D30000AE52C452B7004C225
:10470C0000800B7885E6B405057F0412516DE551E8
:0D471C00700875510AD22A1268457F0522E7
:106D530090053BE0F54E2023037F0522E54ED394B7
:066D63000050F37F0A223C
:105CBE007D077F05124ED6500C7D077F05124ED6FE
:105CCE00503230002F7D017F01124ED65026D22F3A
:105CDE007F0112300A7F011200167D027F07124EDD
:105CEE00D650057F04126EFB9000A0E0FF7C0A7D6B
:0A5CFE00E0125BDE1257197F0F223F
:10602600302337E5484547700C7D087F01124ED670
:1060360050037F372230030EE53A700A126C7B7FDD
:106046000112001680113025037F14227885E6B4EC
:0D60560005057F0312516D7F0F227F14227C
:10234D0090053DE0F54B7F01126EB4126C7B7D0262
:10235D007F07124ED65009E54B70057F04126EE8CB
:10236D009000A1E0FF7C0B7D00125BDED22A12688B
:10237D0045E54570030224777C017D001224F5505C
:10238D00037F3E227C017D501224D550037F3C22D9
:10239D007C017D581224D550037F3C227C017D1099
:1023AD001224DD50081224E550037F33227C017D79
:1023BD00201224DD500B9000BBE0FF7C0E7D408091
:1023CD00207C017D281224ED500512572F80127CA0
:1023DD00017D301224ED50129000B9E0FF7C0E7D8E
:1023ED0000125BDE1267807F00227C017D40D228C7
:1023FD00E4FF1247D4500C7D067F04124ED65003D5
:10240D007F4C227C017D381224F550037F44227CC1
:10241D00017D18C228E4FF1247D4500C7D057F01C1
:10242D00124ED650037F4122E4F55A12570378031A
:10243D00C333CE33CED8F912570CE4FF1247D45024
:10244D001BAF5A1256F1C0071257037805C333CE8E
:10245D0033CED8F9125724D007125B93055AC3E532
:10246D005A648094A840C47F19221224E5500C7D33
:10247D00077F05124ED6504130003E7885E6700438
:10248D007F0180087885E6B404077F0212516D80C4
:10249D00257D037F06124ED6501CE5574556701606
:1024AD009000AFE0FF7C0C7DC0125BDE900532E04A
:1024BD00F556A3E0F5577F19227D077F05124ED6FD
:0724CD0050052000027F050D
:1024D40022D228E4FF1247D422D228E4FF1247D4A0
:1024E400227D077F05124ED622D228E4FF1247D45C
:0924F40022C228E4FF1247D422A1
:106B40003025031267807D077F05124ED650062040
:0E6B500000037F0522900538E0F54E7F1E22DF
:106A1B00E54E70037F23227D027F07124ED650096D
:106A2B00E54B70057F04126EE83023037F0A227F4B
:026A3B001E2219
:106A81001257197D067F01124ED6500C9000ACE0D2
:106A9100FF7C0C7D60125BDE900539E0F54E7F2DA9
:016AA10022D2
:0E6EC2007FA0126EB4900539E0F54E7F2D22B0
:1067F800D22A1268457D027F07124ED65009E54B12
:1068080070057F04126EE8E54E70037F3222302354
:07681800037F0A227F2D22FD
:1061FF00301D037F32227D047F06124ED6501FE5DD
:10620F0055455470199000B0E0FF7C0C7DE0125B97
:10621F00DE900534E0F554A3E0F5557F3222C22F0E
:08622F007F0112300A7F0022FA
:106DB30020210CD221E4FF12055BC2217F00227F38
:026DC3003C2270
:106B5E00202118D2217F40120016D201121D94C29C
:0E6B6E00017F40126EB4C2217F19227F3E22A9
:106E3C0020210A1257391235C4125740227F4122A1
:106E4C0020210A12573912609F125740227F442288
:106E5C0020210A1257391254A0125740227F442283
:05000E0000007F052247
:096F04003024037F0A227F0522DC
:0F6E6C009000A2E0FF7C0B7D20125BDE7F0F22E7
:0F6E7B003024093027037F14227F0F227F142237
:103B6A009000A3E0FF7C0B7D40125BDEE54670030C
:103B7A00023C427D017F03124ED650707C017D08C3
:103B8A00C2287F011247D450037F3F227C017D5017
:103B9A00123C4550037F3D227C017D58123C455022
:103BAA00037F3D227C017D40D2287F011247D450F9
:103BBA000C7D067F04124ED650037F4D227C017D78
:103BCA0028D2287F011247D4500912572F125BDEE0
:103BDA007F00227C017D18C2287F011247D4500C35
:103BEA007D057F02124ED650037F43227D027F035A
:103BFA00124ED65043E4F55AAF5A1257057803C30A
:103C0A0033CE33CED8F912570C7F011247D4501D48
:103C1A00AF5A1256F1C007AF5A1257057805C33387
:103C2A00CE33CED8F9125724D007125B93055AC364
:0A3C3A00E55A648094A840C07F00A2
:093C440022D2287F011247D4228C
:106B7C00202118D221C22F7F0112300A7F01126E00
:0E6B8C00B47F0112055BC2217F00227F3D22F3
:1065430020212A12574712300A7FF47E01126C2A47
:106553007F10120016D202121B93C2027F10126E1A
:10656300B4C22F7F0212300AC2217F00227F3F2252
:1067D00020212212574712300A7FF47E01126C2AC0
:1067E000D2027F011235C4C202C22F7F0212300AC8
:0867F000C2217F00227F432239
:106AA20020211B12574712300AD2027F0112609F27
:106AB200C202C22F7F0212300AC2217F00227F4D02
:016AC20022B1
:1055D400AF5AEF3395E0FE22900520E0F547A3E0B3
:1055E400F54822900522E0F549A3E0F54A2224601B
:1055F400F58274013EAD82FCD2282274702FF582AC
:1056040074003EF583E0FF22C202C2217F192224E6
:1056140050F58274053EAD82FC22055AC3E55A64F6
:105624008094A822D221C22F7F0122D221C22F7FAF
:02563400022250
:10327100E552700612662F8F5222E552B4050612EE
:1032810038A18F5222E552B40B06126A3D8F5222A9
:10329100E552B40A0612439F8F5222E552B40F063B
:1032A100126DC58F5222E552B4110612590F8F5279
:1032B10022E552B412061251E78F5222E552B4149C
:1032C10006120D3F8F5222E552B419061265D28FB4
:1032D1005222E552B41E061265738F5222E552B492
:1032E1002306125EAC8F5222E552B42806126ED02C
:1032F1008F5222E552B42D061261518F5222E552AE
:10330100B432061262378F5222E552B43C06126D76
:10331100D78F5222E552B43D06126C608F5222E5DE
:1033210052B43E061268DA8F5222E552B43F0612B9
:103331006DFA8F5222E552B44106126B038F52226D
:10334100E552B443061269D58F5222E552B44C06B8
:10335100126C958F5222E552B44D061269F88F52C4
:1033610022E552B4370612585E8F5222E552B43923
:10337100061258048F5222E552B438061268FF8FA4
:103381005222E552B43306126A5F8F5222E552B4DB
:0C3391004406126D108F5222E4F5522207
:10662F007D077F05124ED6500D30000A90052AE0E7
:10663F00F52BA3E0F52C7D067F02124ED6500C9061
:0E664F00052CE0F529A3E0F52AD21E7F0522D6
:1038A100302314200F11C21B7D047F01124ED6500C
:1038B100037F0B227F0A22302414201111D21B7D99
:1038C100047F02124ED650037F0B227F0A227F080B
:1038D1001262DD50061245C77F0022202308300FF7
:1038E10005C20F7F0522202408301105C2117F0572
:1038F100227D057F06124ED6501EE53945387018D7
:103901009000B5E0FF7C0D7D80125BDE90052EE01E
:10391100F538A3E0F53980687D067F06124ED65052
:103921001EE53C453B70189000B6E0FF7C0D7DA084
:10393100125BDE900530E0F53BA3E0F53C80417D74
:10394100077F05124ED6500B300008E52C452B7031
:1039510002C2007D067F02124ED65019301E16E5B6
:103961002A45297010C21E9000BCE0FF7C0E7D60CC
:10397100125BDE800B7885E6B405057F0412516D7C
:0F398100E551700875510AD22A1268457F052258
:106A3D0090053BE0F54E202306201B037F05222009
:106A4D002406301B037F0522E54ED3940050E77FCB
:026A5D000A220B
:10439F007D077F05124ED650127D077F05124ED630
:1043AF004003024450200003024450201B3FD22FF1
:1043BF007F0312300A7F0F126EB490000FE0B40229
:1043CF00047F05800990000FE0B403057F01120000
:1043DF00161255DC7D027F07124ED650057F041250
:1043EF006EFB9000A0E0FF7C0A7DE0804E301B51F9
:1043FF0090000FE0FF64026005EF640370437F0FCE
:10440F00126EB47F051262DD400BD22F7F01123086
:10441F000A7F028009D22F7F0312300A7F0A12000F
:10442F00167D027F07124ED650057F04126EFB12C7
:10443F0055E79000A2E0FF7C0B7D20125BDE7F0F23
:0A444F00221255DC1255E77F0F2200
:106DC500201B063023037F1122301B053024027F50
:026DD500122288
:10590F00302352E5484547700C7D087F01124ED673
:10591F0050037F3722300329E53A70257FA0126E9E
:10592F00B490000FE0B401047F01800990000FE0F4
:10593F00B402057F05120016E4F542C21DC20380B2
:10594F00113025037F14227885E6B405057F0312F5
:08595F00516D7F11227F14221B
:1051E700301B1030230D200F0A7F0A126EB4C21B2A
:1051F7007F0A22301B4C302449201146300303120A
:105207006C7BE54A4549700C7D087F02124ED650EB
:10521700037F3822300417E53A70137FA0126EB46B
:105227007F02120016E4F542C21DC2048011302726
:10523700037F14227885E6B405057F0312516D7F3D
:105247001222201B1230240F20110CD21BC22F7FD9
:0A5257000212300A7F0A227F14229F
:100D3F0090053DE0F54B7F0F126EB4201B0C900019
:100D4F00A1E0FF7C0B7D00125BDE301B0C9000A33B
:100D5F00E0FF7C0B7D40125BDEE542B403037F14A2
:100D6F0022126C7BE4F5427D027F07124ED65009AA
:100D7F00E54B70057F04126EE8D22A126845301BCE
:100D8F0003020E82E5457003020E827C017D001284
:100D9F000FFF50037F3E227C017D50120FCF500377
:100DAF007F3C227C017D58120FCF50037F3C227C69
:100DBF00017D10120FD75008120FE750037F332217
:100DCF007C017D20120FD75003020EE97C017D2894
:100DDF00120FEF500C9000BAE0FF7C0E7D20020E38
:100DEF00F27C017D30120FEF500C9000B9E0FF7CC8
:100DFF000E7D00020EF27C017D40D228E4FF1247E7
:100E0F00D4500C7D067F04124ED650037F4C227CAB
:100E1F00017D38120FFF50037F44227C017D18C2E1
:100E2F0028E4FF1247D4500C7D057F01124ED65097
:100E3F00037F4122E4F55A1255D4EF7803C333CE22
:100E4F0033CED8F91255F2E4FF1247D4501D125584
:100E5F00D41255FFC0071255D4EF7805C333CE33E4
:100E6F00CED8F9125613D007125B9312561E40C7F5
:100E7F007F1922201B03020F75E5467003020F75C1
:100E8F007D017F03124ED64003020F2D7C017D089A
:100E9F00C2287F011247D4500F7F50120016D22F55
:100EAF007F0212300A7F3F227C017D50120FDF50EC
:100EBF00037F3D227C017D58120FDF50037F3D22BF
:100ECF007C017D10120FF75008120FE750037F338C
:100EDF00227C017D20120FF750129000BBE0FF7CA7
:100EEF000E7D40125BDE1267807F00227C017D4009
:100EFF00D2287F011247D4500C7D067F04124ED6A4
:100F0F0050037F4D227C017D18C2287F011247D4E8
:100F1F00500C7D057F02124ED650037F43227D0277
:100F2F007F03124ED6503CE4F55A1255D4EF780396
:100F3F00C333CE33CED8F91255F27F011247D450B6
:100F4F001D1255D41255FFC0071255D4EF7805C3A3
:100F5F0033CE33CED8F9125613D007125B931256F5
:100F6F001E40C77F19221210075008121007504158
:100F7F0030003E7885E670047F0180087885E6B4FE
:100F8F0004077F0212516D80257D037F06124ED616
:100F9F00501CE557455670169000AFE0FF7C0C7D56
:100FAF00C0125BDE900532E0F556A3E0F5577F19CE
:0F0FBF00227D077F05124ED650052000027F05C8
:100FCE0022D228E4FF1247D422D228E4FF1247D4BB
:100FDE0022D2287F011247D4227D077F05124ED6DA
:100FEE0022D228E4FF1247D422D2287F011247D4FE
:100FFE0022C228E4FF1247D4227D077F05124ED667
:01100E0022BF
:1065D200C218C22F7F0212300A302505126780804E
:1065E200063027031267A87D077F05124ED6500694
:0F65F2002000037F0522900538E0F54E7F1E2222
:10657300E54E70037F23227D027F07124ED650091A
:10658300E54B70057F04126EE8302306200F037F6E
:106593000A22302408201105D21B7F0A227F1E22E3
:105EAC00201B051255DC80031255E77D067F01127D
:105EBC004ED65024E5427020201B0B9000ACE0FF26
:105ECC007C0C7D60800C301B0C9000ADE0FF7C0CDA
:105EDC007D80125BDE7F2822900539E0F54E7F2D08
:015EEC002293
:0E6ED0007FA0126EB4900539E0F54E7F2D22A2
:10615100D22A1268457D027F07124ED65009E54BBF
:1061610070057F04126EE8E54E601D302306200F96
:10617100037F0A2290000FE06401600930240620A9
:0B61810011037F05227F2D227F3222B8
:10623700301D037F32227D047F06124ED6501FE5A4
:1062470055455470199000B0E0FF7C0C7DE0125B5F
:10625700DE900534E0F554A3E0F5557F3222C22FD6
:086267007F0112300A7F0022C2
:106DD70020210CD221E4FF12055BC2217F00227F14
:026DE7003C224C
:1068DA0020211FC22F7F0212300AD2217F401200CC
:1068EA0016D201121D94C2017F40126EB4C2217FDA
:0568FA0019227F3E227F
:106DFA0020210BD221D202121B9312560C227F3F62
:016E0A002265
:106C600020211512562812300A7F40126EB47F017F
:0B6C700012055BC2217F00227F3D2245
:106B030020211912562F12300A7F10126EB4D201AF
:0F6B1300E4FF1235C4C201C2217F19227F412243
:1069D50020211D12562812300A7F40126EB4D22F84
:1069E5007F0212300AD2027F011235C412560C22E0
:0369F5007F4322BB
:106C950020211412562F12300AD201E4FF12609FF0
:0A6CA500C201C2217F19227F4122A3
:1069F80020211D12562812300A7F40126EB4D22F61
:106A08007F0212300AD2027F0112609F12560C22B6
:036A18007F432297
:106D100020211112562F12300AD202E4FF1254A081
:076D200012560C227F4422F1
:10585E00D20F7D027F07124ED650057F04126EE8DE
:10586E0090000FE0FF64016004EFB4030E7F01129D
:10587E006EB47F401258A77F01801390000FE0B4E2
:10588E00020F7F05126EB47F501258A77F03126E5F
:10589E00E87F50126EB47F3922120016C22E1269A2
:0958AE006CE4FD7F07124F5E223D
:105804003023037F3922E47885F6C20F90000FE03D
:10581400FF64016004EFB4030E7F01126EFB7F404E
:1058240012584E7F01801890000FE0B402147F03D9
:10583400126EFB7F05126EB47F5012584E7F031216
:105844006EE87F50126EB47F0022120016C22E1230
:0A585400696CE4FD7F08124F5E222C
:1068FF00D2117F0A126EB47F40120016D22E126987
:10690F006CE4FD7F07124F5E7F03126EE87F50121B
:05691F006EB47F0022B0
:106A5F0030000B9000B8E0FF7C0D7DE0800C200033
:106A6F000E9000B7E0FF7C0D7DC0125BDEB2007FA1
:026A7F001922DA
:10609F008F5AE55A24FF922E12696CE55A70127FBF
:1060AF0040120016D201E4FD7F09124F5EC201803B
:1060BF0015E55AB401107F10120016D202E4FD7FCD
:0C60CF0009124F5EC2027F50126EB42214
:104D2F00C201C202D20C7F50126EB47F80120016E5
:104D3F0075420390000FE0B401163023647F011217
:104D4F000016302307E542D3940050F67F01804EC2
:104D5F0090000FE0FF64026005EF6403704330239F
:104D6F00267F02126EB4D22F7F0312300A7F0512F4
:104D7F000016302307E542D3940050F6C22F7F026E
:104D8F0012300A7F0580173024177F021200163069
:104D9F00240AE542D3940040033023F37F02126EBE
:0F4DAF00B4E542708E7FA0126EB4C20CC21D22FA
:03000000026BF19F
:106BF100758E0078FEE4F6D8FD9000007FFF7E1FC1
:0D6C0100E4F0A3DFFCDEFA758188024C1080
:103A7E00C2D530F707B2D563F0FF05F030E70CB2D0
:103A8E00D5F4048463F0FF05F080018430D502F490
:023A9E00042200
:103AA000EF8DF0A4A8F0CF8CF0A428CE8DF0A42E3A
:023AB000FE22F4
:103AB200BC000BBE0029EF8DF084FFADF022E4CCF8
:103AC200F875F008EF2FFFEE33FEEC33FCEE9DECC1
:103AD200984005FCEE9DFE0FD5F0E9E4CEFD22ED07
:103AE200F8F5F0EE8420D21CFEADF075F008EF2F51
:103AF200FFED33FD4007985006D5F0F222C398FD42
:053B02000FD5F0EA22DE
:103B0700EB9FF5F0EA9E42F0E99D42F0E89C45F014
:013B1700228B
:103B18007401FF3395E0FEFDFC080808E6CF2FF698
:103B280018E6CE3EF618E6CD3DF618E6CC3CF62271
:0C3B3800A42582F582E5F03583F5832298
:103B4400D083D082F8E4937012740193700DA3A310
:103B540093F8740193F5828883E473740293686024
:063B6400EFA3A3A380DF24
:106E0B00EFC39461400AEF947B5005EF24E0FF221F
:016E1B002254
:00000001FF
